:020000040000fa
:080000000001040000000000f3
:020000040000fa
:10020000afd1200080ff2000000188000000000026
:10021000050007000c000700ca2e020000000000c5
:100220000040da000000fe004440a900c0ad2000fc
:100230000000e0000300320000002000a001880060
:100240004440a800000006006028240001002000af
:100250001600370062004000e080480091018800ed
:100260009001ba0062004000e080480091018800df
:100270009002ba0062004000e08048000002eb00fb
:100280006028e10005003a008301e900070033001f
:10029000038009000059eb00040037006128e100e9
:1002a000010032000082eb00050007009101880088
:1002b0001001ba000200e000e6ff3a00000005006d
:1002c000910188008002780062004000e0804800d0
:1002d0003559ba008301e900080032002559ba00f7
:1002e0008301e900050032000400e000f4ff320061
:1002f00015d9ba008301e900f1ff3a0000000600b9
:1003000000000000000000000000000000000000ed
:100310000000000000000000e1a42000b50007007c
:100320000000e00006003500e1a42000a00020004d
:10033000f60007008000eb000000e00001003d0037
:100340008080eb000100780000000600800078004b
:100350001106b100030035009101b10001003c001d
:100360000050a10000000600040037000204e00075
:100370000a0032000000e8008100e8001041780027
:10038000914f5100f9ff32000081eb0010407800de
:10039000914f500004003900020037000001eb00cb
:1003a0000100370012002000020078000000060063
:1003b000881f7800020478008700070008004000ca
:1003c0004f047800000006000000fa00881f780043
:1003d000000478003fb99700ea8157008000780058
:1003e000801d2000ef000700800078000000e00082
:1003f000020035000040eb0080707c0001007800b6
:100400004f0478000080fa0000000600889fbe00bc
:100410000004be00606380000000e00001003200c4
:10042000000001000800e00001003a00586380006d
:100430000800be0094010700000444001804e00016
:1004400004003a0020cb2000506388000004eb0039
:10045000070037000800be009d01070000004400af
:100460001004e000010032000058eb0050638800e7
:10047000080078004f04be00000006000003b10031
:100480000b0035009000b100080034008000b1007e
:10049000070035005000b10004003400b001b10085
:1004a000030035005000b10001003c0010000500c1
:1004b000000005000200fa00889fbe008a9fbe006f
:1004c0008c1f78008005780001057800020678000e
:1004d0000100e00001003a006c8557000b04780031
:1004e000010037000804e800984478000900fb0088
:1004f000890107000000e000faff3a00d0c2b30013
:1005000080cf54000500320000c0e90080cf5400c5
:100510000200320080447800010037000804e8003f
:100520000c0178008a00780008007800820107003a
:100530000001be009a0f540001003a000b0d780034
:100540009a8f550003003a00e00f5100e08f5900e8
:100550000f003a00b0c2b30080cf540004003a004c
:10056000e00f5100e08f590015003d0008003700f2
:10057000d0c2b30080cf540011003a000000200028
:1005800001002800800f5100818f59000a003600b9
:1005900020022000406388000200200003002800a1
:1005a0006b40400080cf540005003200f2ff2f0066
:1005b000f3ff27000200370060011100e0811900fd
:1005c0000200be004f0678004f05be004f04be007b
:1005d0000080fa0000000600800178000200370069
:1005e000b15978000201e9000200e000fcff3a0086
:1005f00000000600889fbe008a9fbe0000057800ac
:10060000810478002d003700c90090006900900037
:10061000808f50000400390009007800b8020700fc
:100620000000e000350035000040200019006000a7
:1006300009003200a10020000a007800f302070040
:10064000800578000000e000030032000a0050003e
:100650000004e800040037000a007800f6020700f2
:10066000000478008005eb00c9019000690090004b
:1006700003005000880f5000020031000004780091
:100680008005eb00080178008a00780003007800fc
:10069000d1ff070008054500490090000000440014
:1006a000c00498000b00e00004003200090078004c
:1006b000e80207000000e00010003a001a04e00021
:1006c000d1ff3a00008020001900600004003200d1
:1006d00009007800df0207000000e00007003a0090
:1006e00000c02000190060000500320049009000a1
:1006f000e00498000000eb00010037000080eb00f0
:100700004f05be004f04be0000000600889fbe00db
:100710008a1f780080047800010478000045780082
:10072000c100900068009000808f500004003900e4
:1007300008007800720207000000e0001500350094
:10074000480090000958780040049800180078008c
:1007500000b8a30004003a0000a8a300060032007d
:10076000ea4f550004003a0008007800b90207007b
:100770000000e00007003a0000c020001800600000
:100780000200320048009000600498000a80fb00dc
:10079000010037000080eb004f0578004f04be00d9
:1007a000000006006200fa00889fbe008a9fbe001b
:1007b0000004be00020578008300780060f92f0075
:1007c0000f0040007601070088979f0099979f00cf
:1007d0000000eb00a09f9f009a4578000b80fb0073
:1007e0000000ea00cf04de0050c2b30080cf550005
:1007f0000200320009047800010037000904e90012
:100800000800e0000b0034001f90970008017800fa
:100810008a0078008f9197000300010090979f0055
:100820000000e000930032002f9897000000440081
:10083000a09f9f000905450050c2b30080cf55001e
:10084000040032000b04e000e3ff3a002f98970009
:10085000890037000000eb00809f9f00f0979f0009
:10086000e0979f00d0979f00c0979f00b0979f0090
:10087000c09f9f0009003700a0c5200000805000e5
:1008800000004000e1c42000e08078004f9897000d
:1008900001007000c09f9f000a05e8001a4478001c
:1008a0008800fb00a0c520004201070080007800fe
:1008b0000000e000f0ff3a00a0c2b300804f5400f7
:1008c0000e003a00bf8897000180e900b08f9f00ba
:1008d00010007800b09f9f000000e00005003d0080
:1008e0000000ea00b09f9f004f9897000020a000f2
:1008f000c09f9f000a05e80010003700b19f9f00cd
:1009000009003700bf989700f0ff2700808f500044
:10091000040032006a08b9000000410003004000f2
:10092000b09f9f000a05e8001a01fb0003fd2f009d
:1009300003004100e90f5000f2ff3600e0c2b300af
:100940009a4f1000040032000080eb00909f9f003f
:100950008a0478001c0037008a04e800a0c2b300b3
:10096000994f100007003a00bf8897000180e90006
:10097000b08f9f0010007800909f9f008a84e8004d
:10098000110037000000eb00909f9f000900370026
:100990009f989700f0ff2700808f500004003200de
:1009a0006a08b9000000410003004000909f9f00ca
:1009b0008904e8001901fb0003fd2f00030041003a
:1009c000e90f5000f2ff3600194478008800fb0060
:1009d000a0ca2000f70007000000e00002003a0073
:1009e00000447800010037008904e800a87f9f00d8
:1009f00080c6b300804f540004003a00994f1400a1
:100a00000a003a006640500006003700c0c6b30036
:100a1000804f540005003a00994f140003003a003b
:100a200065404000a07f9f008904e8000905e800b8
:100a3000c8fb2f000f04440060f92f000f00400096
:100a40008085e800880178001941780080007800ee
:100a50000b0078003c0207000000e00005003a00af
:100a6000880078000b007800db0007000000e00041
:100a700059ff3d000080eb004f05be004f04be0053
:100a80000080fa0000000600000278000b0037002a
:100a900001017800924178000304e00002003a006e
:100aa000040050000000060083cf52000200320014
:100ab0000201e800f7ff37000000e80090427800ec
:100ac0000504e000f2ff3a000400500000000600b8
:100ad000000278000700370083cf52000a0032007e
:100ae0000201e800924178000304e000faff3a00b6
:100af0000000e800904278000504e00004003200a5
:100b000001017800f7ff37000400500000000600e4
:100b100004005000000006006900e10004003500f8
:100b20006d00e100030034000002b100010032005a
:100b30000000050010000500ec874700889fbe00fc
:100b40008a9fbe008c9fbe008e1f7800f0b79f006a
:100b500081bf9f0082047800000478000100370004
:100b60000804e800184778000e00fb00eaff0700c1
:100b70000000e000faff3a00d0c2b300804f5700f7
:100b80000500320000c0e900804f5700020032002b
:100b900000477800010037000804e8000900e00081
:100ba00045003500e18f5400430032004002200030
:100bb000808f540040003c000900e0000e0034002b
:100bc000f08f54001a003a0000c3b300984f100091
:100bd00016003a009840900080c7b30080cf5000c4
:100be0000300320080c5b30080cf50000f003a00f0
:100bf0000884e8000e003700a900200000c3b300fd
:100c0000984f10000a003a009840900080c7b30047
:100c100080cf5000040032008900200080c5b3005e
:100c200080cf500002003a000884e800090120004b
:100c300008057800010037000a05e80000c3b3008a
:100c40009a4f1000fcff32008a0578006066b800f9
:100c50000e00370090b4200000425200c4ef9f0005
:100c60006149b9000c00be001b0a07004fea97005b
:100c70000401fb00cf91de008b05e800ccb79f009c
:100c8000ddb79f0000064100818649001b00fb0084
:100c90002b030700800078000901780090b4200041
:100ca0002e030700000278000000e000e9ff3a0090
:100cb0008b0f540006003a000fb897000000e000c8
:100cc00029003200ffb097000108780026003700a5
:100cd0008a80550040b22000694078000000fb0087
:100ce00000805000160033004240a9000f003c0075
:100cf0004fe997000200fb00cf80de0000005600a5
:100d000081805e00800f5600818f5e0007003900f1
:100d10006149b900f60907004fb19700dfb19700ac
:100d2000820f5000838f58000500320020022000ff
:100d3000406388000086eb008086eb0005003700ea
:100d4000d0c2b300804f570002003a006006160080
:100d5000e0861e008fb997000300e0000300320018
:100d60008b097800010037006066b8000c00be00f7
:100d70004f0778004f06be004f05be004f04be006f
:100d8000cf00b10000000600306380000000e000ea
:100d9000010032000000010080c6200000000600b3
:100da0000200fa00f1bf9f00010878000080fa00fd
:100db00000000600040037000204e00001003a00d1
:100dc000000005000000e80010417800814f51004c
:100dd000f9ff3a00000006000400fa00889fbe00f8
:100de0008a9fbe008c1f78000004780001067800fe
:100df00070089000f80090000100500088089000f2
:100e0000010050009808900001005000a8089000d0
:100e100001005000b808900001005000c808900080
:100e20008105500000022200a0bf9f0000032300a4
:100e300090bf9f00081090000028a30018003a00ff
:100e40000b00e000160034008b04780009057800e0
:100e5000e28f5400020036002a0020000200370012
:100e60000900e0000b00340058009000c801900019
:100e70000a017800ec80570003000100500498003c
:100e80000000e00096003200680890000000450075
:100e9000600c98008a8454004240a900ebff3c009b
:100ea000780190000200e0000b0034005800900030
:100eb000c80190008c0078000300010050049800e5
:100ec0000000e0008600320068089000f800900002
:100ed00001004000600c9800880c90000900e000c0
:100ee0001500340009057800e28f54000200360036
:100ef0002a002000020037000900e0000b00340047
:100f000058009000c80190000a017800ee80570058
:100f100003000100500498000000e000700032005f
:100f20006808900000004500600c98008a84540016
:100f30004240a900ebff3c00180990000200e000cd
:100f40000b003400e800900058009000c8019000a9
:100f500003000100500498000000e000600032002f
:100f6000680890009808900001004000600c98000c
:100f7000a80c90000900e000150034000905780075
:100f8000e28f5400020036002a00200002003700e1
:100f90000900e0000b00340058009000c8019000e8
:100fa0000a017800ee805700030001005004980009
:100fb0000000e0004a003200680890000000450090
:100fc000600c98008a8454004240a900ebff3c006a
:100fd000380990000200e0000d003400e8009000a5
:100fe000180890008080400058009000c8019000d0
:100ff00003000100500498000000e00038003200b7
:1010000068089000b808900001004000600c98004b
:10101000c80c90000900e0001500340009057800b4
:10102000e28f5400020036002a0020000200370040
:101030000900e0000b00340058009000c801900047
:101040000a017800ee805700030001005004980068
:101050000000e00022003200680890000000450017
:10106000600c98008a8454004240a900ebff3c00c9
:10107000081090000028a3001b0032000b00e000c5
:10108000190034008b04780009057800e28f5400c1
:10109000020036002a002000020037000900e000ac
:1010a0000b00340058009000c80190000a0178003d
:1010b000ec80570003000100500498000000e0009d
:1010c000070032006808900000004500600c98009e
:1010d0008a8454004240a90003003400eaff37002c
:1010e0000080eb00010037000000eb004f067800a5
:1010f0004f05be004f04be000080fa00000006004d
:10110000889fbe0000047800c0019000600090003d
:101110008000eb00808f5100390039001801780001
:101120002000290000006100e20f5000070032009b
:10113000002020000200e000010035000020240013
:10114000000c71008080eb002d00370001002600ac
:1011500001006100810f500008003a003800900043
:10116000808f510005003900080078003900070021
:101170008080eb000000e00021003a0000c0200069
:101180001800600017003a00a804900060022000d8
:1011900008004000808f540012003a000020200018
:1011a000e102070080007800200498000000e000c1
:1011b00005003a0029049800490498000900e80055
:1011c00030049800060037001860a0004004980022
:1011d0000020b00030049800410c9800510c980099
:1011e000fe0207002800900050049800380090008c
:1011f0006004980000002600180c70008000eb00ce
:10120000010078004f04be00000006008001eb00e2
:1012100010417800814f510001003a0080017800b0
:101220000204e000020032000000e800f8ff37008e
:1012300003007800000006008000780001003700fd
:101240000000e8001004e000fdff3a00010050003b
:1012500000000600889fbe00000478000000e00047
:101260000e003a00800478008980440060a12000cc
:10127000610078000000e00004003200f5ff070084
:101280000000e00001003d000084eb008904e8005c
:10129000e78f540029003c00f3ff370000002200d4
:1012a0001800600024003200a804900008003700f5
:1012b00009015000384090000000fb0089007800d0
:1012c000c50707000000e0001300340080844400dc
:1012d00048009000808f5400f5ff390028009000ee
:1012e000400498001801780000c020000000610050
:1012f00002003200a800900001003700b800900002
:1013000000002400000061000a003200610498001f
:101310000004eb000900370028009000400498000a
:1013200060049800500c98001890a0000084eb0016
:1013300002003700510c9800000478000800780083
:101340004f04be0000000600889fbe008a1f780080
:1013500000047800010278008244780003057800d8
:1013600070c6b300804f510021003c0000c0e9006e
:10137000804f5100df003d0072405000804f51000f
:101380004c0132000d003c006c405000804f510079
:101390005f013c0000c0e900804f5100d5003d00d6
:1013a00050c2b300804f5100560132007c404000d3
:1013b000804f510056013a00ce00370010c6b300ee
:1013c000804f5100cb00320004003c0069405000c7
:1013d000804f51004e013a007200370030c6b30012
:1013e000804f5100180032000040e800090037002b
:1013f00000c7b300804f51001f01320008003c00bd
:1014000000c0e900804f5100e500320065003c005b
:101410006540500080cf54003d013a000f00370076
:1014200050c7b300804f51005e003200634040005f
:10143000804f51005b00320065405000804f5100ea
:1014400033013a001b0137009180e900010a78005e
:101450007800900011f0790033013700a860900007
:10146000c0c6b30080cf50000a003a009400780054
:1014700064805000000a78001000be004f89de0032
:10148000cf91de000002be000203780082037800e4
:101490001300370010c7b30080cf500003003200a4
:1014a000a0c6b30080cf500006003a009400780038
:1014b00068805000000a78003002be002003be00a1
:1014c000070037001480e900000a78001000780057
:1014d00000027800cfa2de000503780086037800c2
:1014e000049cbe000694be00a860900080c6b300b5
:1014f00080cf50000e00320020c6b30080cf5000d5
:1015000005003a000400fb00cf80de0001017800f6
:10151000820178000a00370040c7b30080cf500036
:10152000030032006640400080cf500006003a00c1
:1015300004007800cf80de0001017800820178008d
:10154000009cbe000294be003800be002801be0010
:10155000e00f5000e08f5800e00f5900e08f590075
:1015600003003d0078009000d1c2b3000a003700ac
:10157000081090000018a3000300320078009000cb
:10158000b1c2b300040037000008a30054003200c9
:101590007800900001c2b30001707d000000e800f7
:1015a0004e003700a8609000c0c6b30080cf500046
:1015b00007003a009400780064805000000a780028
:1015c0001002be000003eb00860378001300370012
:1015d00010c7b30080cf500003003200a0c6b30094
:1015e00080cf500006003a009400780068805000d8
:1015f000000a78003002be002003be00070037005a
:101600001480e900000a78001000780000027800d9
:10161000050020000600200007002000049cbe00fa
:101620000694be00a860900080c6b30080cf500032
:101630000e00320020c6b30080cf500005003a00f3
:101640000480fb00010020000200200003002000b5
:101650000a00370040c7b30080cf500003003200bb
:101660006640400080cf500006003a000400780039
:10167000010020000200200003002000009cbe00aa
:101680000294be00081090000038a300140032003d
:101690003800be002801be00e00f5000e08f580067
:1016a000e00f5900e08f59000d00320080c7b300f1
:1016b00080cf54000300320080c5b30080cf5400b7
:1016c00007003a007800900001c3b30001707d006c
:1016d0008000e80089707d000080e80070049800b8
:1016e0007800900000004500600498008940780070
:1016f0006d003700a8609000c0c4b30080cf5000d8
:1017000006003a009400780068805000000a7800d3
:101710005001be004000be00050037009400780074
:1017200064805000000a78001000be0080070700a7
:10173000009cbe000294be00380090000000e00053
:1017400003003d0078009000d1c2b3000a003700ca
:10175000081090000018a3000300320078009000e9
:10176000b1c2b300040037000008a3000500320036
:101770007800900001c2b30001707d000000e80015
:101780007004980078009000000045006004980004
:101790008940780008007800e30107006400370002
:1017a000a8609000c0c6b30080cf50002500320072
:1017b0000a003c006440500080cf500028003200f6
:1017c00000c0e80080cf5000140032006840500094
:1017d00080cf500022003a000a00370040c7b30013
:1017e00080cf50001e0032006640400080cf500085
:1017f0001b0032006940500080cf500018003a00b2
:10180000060037001480e900000a78001000780014
:10181000485c900008487800450037001480e900d3
:10182000000a78001002780068089000cf80de007f
:101830000101780082017800009abe000292be0089
:101840003b0037001480e900000a7800100178009e
:1018500068089000cf80de000089be0034003700a9
:101860001480e900000a780010007800680c9000ed
:10187000080878002e0037001180e9008008780001
:1018800010007800cf80de0001017800820178002e
:10189000009cbe000294be0078009000000045004d
:1018a0006004980081c7b300080078003600070084
:1018b0001f0037001480e900000a7800100078004b
:1018c00060049800580990000200e00002003d000a
:1018d00059fe0700090037008000eb001f000700d9
:1018e000800078000000e0000300320068009000f3
:1018f000008050000100370058089000100c98003c
:101900000b0037007800900002707d000600370061
:1019100078009000800045000904e00001003a00d2
:1019200059c2b300894878000000e80070049800ac
:101930000000eb004f0578004f04be0000000600d9
:10194000800078001104b100030035009101b1005e
:1019500001003c000050a000000006000600370017
:1019600090cf100002003a00000178000400370018
:101970000000e8000201e9000200e000f8ff3a0080
:101980000200780000000600ef02b000889fbe0051
:101990008a9fbe008c9fbe008e1f78008006780054
:1019a00000012000b0b79f00d2c32000c2b79f0043
:1019b00080c5b30080cf50000e00320083002000ad
:1019c000b3b79f00c4c22000c4b79f007740400057
:1019d00080cf50000700320000012000b0b79f0008
:1019e00080c7b30080cf500002003200a200200068
:1019f000b2b79f003d04be002d05be0040c6b30037
:101a000080cf5000030032006540400080cf50007e
:101a10000b003a00e00f5400e08f5c00e00f5d0027
:101a2000e08f5d0006003d006000b8006011b80066
:101a300008045000898458000a0559008b85590014
:101a4000e00f5400e08f5c00e00f5d00e08f5d0070
:101a500004003a005d0890008e0120000000e000c4
:101a60000c003200bfb1970003027800cfa2de0065
:101a700005037800860378000800be000a01be0056
:101a8000530707004fb2970064407800d0df9f00f3
:101a90007e0120003fb0970000027800cfa2de0058
:101aa00005037800860378000800be000a01be0026
:101ab0004007070023003700bfb0970001047800fb
:101ac000cfc4de00090578008a0578000802be0050
:101ad0000a03be007fa897008fb097001fb1970040
:101ae000afb197003e070700d0b79f00e1b79f0056
:101af000f2b79f0083bf9f000e07e90062fc2f0032
:101b00000f014100020647000802be000a03be00a2
:101b10005fb09700efb097007fb197008fb9970043
:101b20001d0607007faa970000005200cfb0970063
:101b300060ce78005fb09700efb097007fb197005c
:101b40008fb99700809ebe008296be003d00be0009
:101b50002d01be00f0af9f0081b79f0092b79f009c
:101b6000a3b79f00e00f5000e08f5800e00f59002e
:101b7000e08f5900020034000e00e000ceff3c0070
:101b8000bfb09700e88f500010003a000d10900091
:101b90000038a3000d003200f70f570006003e008a
:101ba00062fc2f000f0141008200470000c3b30018
:101bb000914f1000050032000e07e90000c3b3008a
:101bc00063fc2f008e81410080f17f0078011700b7
:101bd000920e98006d00900063fc2f008f814100f1
:101be0008e8041007cfa07001d0990005d0890007e
:101bf000800f510006003d0002005000800e98004a
:101c00000d1090000040a100801698000f003700d2
:101c10000000e0000d003d000d1090007400600019
:101c2000f00f500009003a007d089000fd00900080
:101c3000010050008d08900001005000020050008b
:101c40004240a90001003400800e98004f07780040
:101c50004f06be004f05be004f04be00ef02b100ac
:101c600000000600889fbe00800478001263800098
:101c70000200e00002003200020078000c00370091
:101c800040c6200003003700918f54002400360026
:101c90000180e800900078000100e000faff3a00bf
:101ca0000f003700918f54001d0036000180e800be
:101cb000900078000100e000faff3a00120178007d
:101cc00040c6200003003700918f540014003600f6
:101cd0000180e80090007800828f5000faff3a00ff
:101ce00008638000890f5400010031000904780066
:101cf00008007800aa0207000000e00004003a0093
:101d0000890f5400050032000804d100f5ff3700a8
:101d100008187800a9020700d4ff37000000eb0084
:101d20004f04be0000000600881f780063044000d6
:101d30000800a100800f540023003600e30f540078
:101d400001003e004800200008007800c5ff0700a1
:101d5000800078000000e0001b00320010017800d5
:101d60009201780064805100880f50000300310018
:101d7000120090008008780007003700080041003a
:101d800080087800920190001300980011007800fc
:101d90001208140008097800910078000100e000a2
:101da00005003200110090000000e0000200320047
:101db0000180e800010037000000eb00106388009c
:101dc0000280e800010037000000eb004f047800bb
:101dd00000000600c0f72000ab0237006e4ce200a6
:101de00003003a00fbff070020c0b3006eecb70011
:101df00000000600889fbe000004780015fd070063
:101e00008004780000042000180060000200320006
:101e100028009000690207000000eb0020049800f1
:101e2000384090000004e000050035000000fb0091
:101e30001f0507000000e000010032008084eb0075
:101e4000181090000000e000080032002305070091
:101e50000000e000010032008084eb0018109000c8
:101e6000560207000000eb00101498000008200044
:101e7000180060000f0032008000eb00018140007c
:101e800063a1200062807900880f500006003200b4
:101e90008100e800e78f5000f8ff36000800780066
:101ea0004602070011003700030041000008eb0064
:101eb000faff3700000c780000c0eb0030449800b7
:101ec00060022000080040002004980040049800b0
:101ed00050049800400c980060049800500c980042
:101ee0007004980076004400000c98000900780007
:101ef0004f04be0000000600881f78007800200014
:101f00008800440060a12000610078000000e0002b
:101f100001003200b7ff07000804e900f8ff3b00aa
:101f20004f047800000006000f04b000889fbe0038
:101f30008a9fbe008c9fbe008e1f7800f0b79f0066
:101f400081f79f005001be004000be00b09f9f007f
:101f5000c19f9f00d29f9f00e39f9f0010c6b300c8
:101f60000ff19700804f51001600320010c4b300eb
:101f7000804f510013003200ffb1970053089000ca
:101f80000000e00003003d0060002000d009980040
:101f90000c0037000000e0000a003a0070c6b300f1
:101fa0000ff29700804f52000300320070c4b3005c
:101fb000804f520003003a0010002000ffb297004b
:101fc000d00a9800ffb0970040fb2f000f004000a0
:101fd0003a02070080017800e20f500015003a0035
:101fe00030002000ffb097009008980010c6b300a2
:101ff0000ff19700804f51000a003200644040000a
:10200000804f5100070032000040e800804f51002f
:102010000400320081c720000040e800804f5100da
:1020200001003a00c1c72000ffb197006300900093
:10203000160037000000e0001800340030002000d7
:102040007fb29700100a980010c6b3008ff2970075
:1020500080cf52000a0032006440400080cf52001e
:10206000070032000040e80080cf52000400320038
:1020700001c820000040e80080cf520001003a0073
:1020800041c820007fb1970062009000315878006d
:102090003158780011487800bb01370014c6b300ee
:1020a0008ff2970084cf52000300320010c4b300b7
:1020b00080cf520013003a007fb09700600190007b
:1020c0008200780000c3b30080587800ffb2970008
:1020d000e102980080c7b3008ff2970084cf5200ce
:1020e0000100320080c5b300804878000280e8001b
:1020f000ffb09700e0009800710090000080e800b9
:10210000f00098000300e00005003a00a39f9f0044
:10211000e4fb2f000f014200030778009501370010
:1021200085c82000e5b79f0010c6b3008ff0970068
:1021300080cf50000500320010c4b30080cf5000a3
:10214000a0003a0092c92000e2b79f00ffb19700bb
:10215000530890001e0220000000e000010035003e
:102160000007e8000e02e800d4b79f006022b80024
:102170006033b8003f989700cf9897005f99970019
:10218000ef99970012060700ffb097003102be00da
:102190002103be000000e00004003d000400be007a
:1021a0000601be0003f0a200020037000400be00da
:1021b0000601be00b09f9f00c19f9f00d29f9f005d
:1021c000e39f9f002f99970064015100a29f9f00f9
:1021d00043fb2f008f8141006a8041000048eb00e3
:1021e0006b824100c4b79f0031003700c20120005c
:1021f0000300200065fb2f000f804200db01070079
:102200003f9c9700cf9c97005f9d9700ef9d9700a4
:102210000800be000a01be00f20507000006be006d
:102220005fb1970067015100d2b79f004240a900fb
:102230000a003400170607000002be000203be00b9
:102240000800be000a01be0015060700b09f9f00ef
:10225000c19f9f00d29f9f00e39f9f00cfb1970037
:102260006780410071002000060037000000e9008f
:102270006f4866004c6add004466de000c067200a2
:10228000c4eede00e00f5600e08f5e000400340074
:102290008100e900f5ff3b00010037000060eb0022
:1022a0008100e900fdff3b0067004000c0b79f00d0
:1022b000dfb297000500e000090034006022b8009a
:1022c0006033b8003f989700cf9897005f999700c8
:1022d000ef999700f40507000000e000c3ff3c0001
:1022e000e0fb2f008f0040004fb19700010051002c
:1022f0000000e9008e0f500001003d00000778004b
:102300000e00e00003003d00f3fb2f000f814100b1
:1023100025003700800f570005003d0001004700f1
:1023200010409000f4c0b300e74f500001003c00a3
:102330000042eb000e007800010037000e07e900b4
:102340000000e900f5fb2f000f81420080014100f1
:102350009340780084cf5000f8ff3200ef4f5200d6
:1023600001003a008149e8000000e00006003d005d
:102370000e07e8002f98970064004000a09f9f0080
:10238000e1fb2f000f8140008e0178000400370030
:10239000830041001100fb006fb29700e0487a0013
:1023a0008301e900faff3b00ffb297005508900057
:1023b0000000e000ef003d000e00e900d00a9800a8
:1023c000ec0037003f9c9700cf9c97005f9d9700e3
:1023d000ef9d97006022b8006033b8000800be008f
:1023e0000a01be007a0507000000e00005003d007c
:1023f0000bf0a200b89f9f00c99f9f00da9f9f002b
:10240000eb9f9f002f989700725927000280b90018
:10241000026a280013002000a8050700e40050000d
:10242000a19f9f0019003b00e3801000c0ff2f0018
:10243000008460000800ea00a09f9f00e9b6200029
:102440000f0037000808a3000b0032003902be005d
:102450002903be003f989700cf9897005f99970097
:10246000ef999700a4050700b09f9f00c19f9f00b0
:10247000d29f9f00e39f9f000884d100e88444001e
:102480000800e000efff3c001f0037000100e00003
:102490001d003400c0ff2f0000806000a09f9f003f
:1024a000000478006000b8000200200003ff230051
:1024b000e9b62000070037000808a3000300320037
:1024c0003902be002903be008b0507000884d10035
:1024d000e88444000800e000f7ff3c000002be0072
:1024e0000203be003f989700cf9897005f9997002e
:1024f000ef999700f5050700b09f9f00c19f9f00cf
:10250000d29f9f00e39f9f00ffb09700510990006a
:1025100060c6b3008ff1970080cf510004003200f5
:102520006100200060c4b30080cf510002003a0077
:102530002f9a9700ea00420001074100f30f57006d
:10254000010034003e01200000c3b300e07f9f0083
:10255000f5fb2f008f824200b5b79f002e00370099
:102560000800be000a01be001e0507000006be00ee
:10257000680757004240a9000e00340045050700d7
:102580000002be000203be000800be000a01be0039
:10259000430507006022b80046782d007719240013
:1025a00055050700b09f9f00c19f9f00d29f9f00cd
:1025b000e39f9f003fb0970068044000890020001f
:1025c00008003700a2002000030020000c00be001d
:1025d0005f0107000804e90004c3b300044c410094
:1025e0000006be00e00f5600e08f5e0006003400db
:1025f0008904e900f3ff3b00030037000804e90009
:1026000000c3b300004c78008904e900fbff3b00e5
:1026100068044400b8b79f000e00e0000b003400cf
:102620003f9c9700cf9c97005f9d9700ef9d970080
:102630006022b8006033b8000800be000a01be0086
:10264000190507000000e000c5ff3c0045fb2f0016
:102650008f8242006a804200bfb097000080500025
:102660000002e9002f99970067014100a29f9f0097
:102670006b814200050037000402e900af99970022
:102680008301e900a39f9f000201e80000c3b3009b
:10269000924f1000f8ff3200ffb29700d50990006a
:1026a00060c6b3008ff0970080cf50000300320067
:1026b00060c4b30080cf500003003a00af9a970087
:1026c0008500e8000a00370050c6b3008ff097007d
:1026d00080cf5000050032008000eb0050c4b300f2
:1026e0008ff2970080cf520001003a0011002000c5
:1026f000018741008e0f520001003d000407780061
:102700000e00e0001b003500840f570005003d005f
:10271000ee40790095c3b30040c3b30080cf5000b2
:1027200001003c0005c3b3008e00780001003700b3
:102730000e07e9008100e9000102410094417800a0
:1027400085cf5100faff320090c3b30080cf520012
:1027500001003a00034ae8000100e00005003d00e6
:102760000201e9000e07e8002f9897000000e8003a
:10277000a09f9f002f9a97008e0178008ff09700fe
:102780007fb097000c0107004f0778004f06be008e
:102790004f05be004f04be000f04b100000006004c
:1027a0000000e00003003400d6020700e10f400003
:1027b00001003a000000eb00000006000000e0000d
:1027c000300032008080e90091027800e38f5200ef
:1027d0002c0036000508a3002a003a00226380007e
:1027e0000200e00002003200828f5000040031003d
:1027f0000208780021638800160037000301780082
:10280000920190000300e00002003200818f51002d
:10281000faff39001202780004004100808f500056
:1028200018003900810f500003003a0005094200ea
:1028300082007800070037000300e0000300320048
:1028400005804000808f51000e00390093009800f1
:1028500011019800110190000200e000090032000f
:1028600011804000820f500006003a00622cef00f9
:1028700011009000110178009008410010009000b4
:102880009000980000000600000178000000200081
:102890000000e00008003200000080000000e000be
:1028a000050032000000e900000088000000400040
:1028b0000100800002b0780000000600889fbe0082
:1028c000800478006684400000ff27001800600044
:1028d0004401de00f07f2000800f51000e003a001e
:1028e000800ceb00180478006f0064001c003a00b4
:1028f000210090000000e00019003a001100900053
:102900000000e00016003a00100020001100e00076
:1029100014003200120037000200e00005003c0005
:1029200001007800d3010700000178000000e000fa
:1029300008003c00f00028001800600001fe2300a1
:10294000010c700020c02f00800c41000080eb00c3
:1029500004003700800ceb000000eb0001003700a2
:10296000200020004f04be0000000600889fbe002b
:102970008a1f78008c9fbe00000478000206be000b
:10298000e6044000190178000200d0004505de0091
:102990008a007800f07f2000800f55000c003a007c
:1029a0006f00610065003a00280090000000e00020
:1029b00062003a00180090000000e0005f003a005a
:1029c000100020001800e0005d0032005b003700be
:1029d0000a00e00007003a0008007800a50107009f
:1029e000800078000000e000020034000a00780057
:1029f000530037006108b9000c0140008d81480088
:102a0000e07f2000800f5100e08f59000d0034005e
:102a10001900e00004003d006000b8000200200042
:102a200003ff2f00030037006000b8000200200001
:102a300003ff2700009cbe000294be00100020008f
:102a40003f003700e00f5100e08f590005003400cf
:102a5000f000280019006000c410dd00810c700037
:102a600034003700190078000100280001036000dd
:102a70006f0060000040a000800c780061015100f0
:102a8000e0815900c0fc2f00f1ff2f00800f5100a2
:102a9000818f59000d003d00860c78000000eb008e
:102aa0002004980010049800000c780024003700df
:102ab0008880e800110c78006400440090087800d9
:102ac00019087800800ceb0070014100f00f410004
:102ad000f7ff34008202ea00150032008881e80026
:102ae00070821200980078008508de0013007800dc
:102af0000400dd00008c7000640144009300780045
:102b00008508de00120078000400dd008089700076
:102b1000920078008508de00190078000400dd00ce
:102b200000897000190078000500de00800c780034
:102b3000990c73000080eb0001003700200020009a
:102b40004f06be004f0578004f04be00000006008f
:102b50000800fa00889fbe008a9fbe008c9fbe00be
:102b6000e0b79f00f1b79f000206be00d303070045
:102b700080bf9f0091bf9f000001be000c00be00ff
:102b8000550207006fb19700ffb197000005510093
:102b9000818559000fbc97009fbc97000800be00bc
:102ba0000a01be004f06be004f05be004f04be0026
:102bb0000080fa00000006000a00fa00889fbe00ac
:102bc0008a9fbe008c9fbe000004780001457800fb
:102bd0000206780083047800840678000300e00091
:102be00002003c00190020004ccb200060c6b3005e
:102bf000804f55000e00320060c4b300804f550076
:102c00000b00320070c6b300804f55000300320045
:102c100070c4b300804f55009c003a00e48f46001a
:102c20008000350058089000808f56007d003d00e0
:102c30008d05e80060c6b300804f550010003200db
:102c400060c4b300804f55000d00320008109000a2
:102c50000038a30004003a0058089000808f540008
:102c600001003d00590c9800580890000b005000de
:102c7000500c980002003b000000eb00500c980044
:102c80000b00e00027003c0018099000680090004d
:102c900001c3b300017178008201e800130c9800b1
:102ca000580890000000e00003003c00081090006d
:102cb0000038a3000500320068009000e1c2b300b4
:102cc000817178000280e800100c9800d80890000c
:102cd0000b00ea00808f500001003d008105ea00f2
:102ce0000b00ea00200c980001804500500c980071
:102cf000890f500001003d0080047800390c9800d5
:102d000068009000980890000100400009017800d8
:102d10008c00780030f60700580890000900500039
:102d20001a00370098089000680090008b8f5400bc
:102d300018003d0001004000090178008c00780077
:102d400025f607001808900000814400120c980036
:102d500009805500200c9800580890000000e00001
:102d600003003c00081090000038a3000600320069
:102d7000e8009000e0c2b30000f17800380890004d
:102d80000000e800300c980058089000400c9800b3
:102d9000a1003700010040000b0178008c00780092
:102da0000df607001808900000814500120c9800ed
:102db0008b845400580890000000e00003003c00a1
:102dc000081090000038a300050032006800900051
:102dd000e1c2b300017178000200e800100c980015
:102de00058089000890f500001003d0080047800d1
:102df0006800900098089000010040008b00460099
:102e000009017800f4f507001808900000804400dc
:102e1000100c98005808900009005000200c9800f1
:102e20007d00370070c6b300804f550003003200ac
:102e300070c4b300804f550014003a005808900049
:102e4000808f540004003d00081090000038a3005b
:102e500001003a00590c9800580890000000e90061
:102e6000500c980002003b000000eb00500c980052
:102e700070c6b300804f550002003a005ac6b30036
:102e80000b0037005ac4b3000900370010c6b30066
:102e9000804f550002003a000ac7b3000400370013
:102ea00010c4b300804f550001003a000ac5b300ba
:102eb00018099000680090003c7178008201e800d9
:102ec000130c98000c027800580890000000e000f5
:102ed00003003c00081090000038a30017003200e7
:102ee000e8009000e0c2b30080f178008280e80042
:102ef000110c9800580890000000e0000f0034000a
:102f00008904e900890f500001003d008004780029
:102f1000680090000080400009017800840078007b
:102f2000adf507001808900000804400100c9800d0
:102f30005808900009005000200c9800680090008c
:102f400098089000010040000086e8000a587800c8
:102f5000800078000d00e00004003500b0c2b3002e
:102f6000804878008c04780004003700d0c2b30099
:102f7000804878008c0478008d06ea008005eb001c
:102f800007003700a10020000d0078008500070031
:102f90007681550001f17f008b05e80080067800fe
:102fa0000d00e000f7ff3c00e18f55000e003c00f3
:102fb00050c6b300804f55000300320050c4b30028
:102fc000804f550003003a0000c3b300005e780054
:102fd0008c0478000b00e00008003a0000c3b30046
:102fe000805c7800070037008b05e900f680570009
:102ff0000180450002c3b300905c41000b00e0007b
:10300000f9ff3c0068009000980890000100400023
:1030100000805400300c980008109000740060008c
:10302000f00f50000e003a007800900098089000d1
:1030300001004000a808900001004000b80890007e
:1030400001004000c808900081004000780890000e
:10305000808f500002003d0001005000000c9800dd
:103060004f06be004f05be004f04be000080fa00b0
:103070000000060000027800e6024000150078001b
:1030800001002800810360006f006000800a780062
:1030900012003a00240090000000e0000f003a0007
:1030a000140090000000e0000c003a001600200020
:1030b0001400e0003800320008003700e40042004d
:1030c000910a78000480e8009008780014087800dd
:1030d000000aeb00700353000100370016002000c7
:1030e0001500e000f5ff32001300370064014200d4
:1030f00080004000120078004f00de00808a7000df
:103100008481e800920078008180400013007800fc
:103110004f00de000089700093007800818040003d
:10312000140078004f00de008089700014007800e1
:10313000000a40000603e90015007800ef0f500078
:10314000eaff3600100037000481e8009400d10047
:10315000120078004f00dd00008a7000e400420099
:103160009201d100110078004f00dd00008971004c
:103170001101d100150078004f00dd0080087100ba
:10318000950ad1000603e80015007800ff0f5000f3
:10319000edff3e00ef0a6000958a7300060078009c
:1031a0000000060001017800801f7800110009006e
:1031b0000200d800800078004f0078000191b9002b
:1031c00082025000010278000400be0000000600e8
:1031d00000c0da00000006000a00fa008001780052
:1031e00081027800e20f500024003e00a0638000be
:1031f000e10f500008003200e02120000000e00054
:10320000050032006321200084212000a621200037
:103210008000780004003700c3202000e420200054
:103220000621200041212000134090000004e0000e
:10323000030035008008eb000000280093097000af
:10324000144090000028a30001003a0014a0a00040
:103250008200780006003700144090000008a300a8
:10326000fdff32003500fb00000b78008100e90013
:103270000100e000f8ff3a00080037006a805700bc
:1032800031002000b1bf9f00c3bf9f00d5bf9f008a
:10329000e2bf9f00ceff07006fb9970002007800e1
:1032a0000080fa000000060000c0da0000000600fe
:1032b0000a00fa0011002000b1bf9f00c0bf9f00ac
:1032c0006a805700f8ff07004fb897000080fa00a7
:1032d0000000060000c0da00000006000a00fa0044
:1032e000800078006a80570052002000b2bf9f0023
:1032f000c1bf9f00f7ff07005fb897000080fa008a
:1033000000000600889fbe0080047800760ce20072
:1033100004003a000000eb00100007000000e0008d
:103320000a003500b06380000900e00002003a00a6
:10333000000478000600370000047800090040000f
:10334000060007000000e00001003d000084eb00e3
:10335000080078004f04be000000060080007800de
:103360000000e00004003a0060cb2000b063880059
:1033700001017800060037000081eb00a0d1200099
:10338000808f500002003e00b16388000001eb0016
:103390000200780000000600889fbe008a9fbe00e1
:1033a0008c1f78000205be000004be000006eb0082
:1033b000e00f5000e08f5800e00f5900e08f5900f7
:1033c00007003d006000b8006011b800080450001c
:1033d000898458000a0559008b8559001c0020007b
:1033e000e00f5200e08f5a00e00f5b00e08f5b00bf
:1033f00002003d000f0007000c00a2000800be0004
:103400000a01be00120007000203be000002be0057
:103410000c00e00001003200060007000400be00be
:103420000601be004f0678004f05be004f04be00e7
:10343000000006006000b8006011b80004025000ef
:103440008582580006035900878359000000060052
:10345000889fbe008a9fbe008c9fbe000404b800f7
:103460000506b8008904460060854e000606b800cf
:103470000a054600e0854e000706b8008b054600a9
:10348000040eb800890446000a854e00e0854d0010
:10349000050eb8000a0546008b854e00060eb800e2
:1034a0008b0546000416b8000a0546008b854e00c1
:1034b0000516b8008b054600041eb8008b054600b3
:1034c0000800be000a01be004f06be004f05be0048
:1034d0004f04be0000000600020ab900001bb9003c
:1034e0000200b80081004200810043000000060095
:1034f0006022b800060220000000d0008180d200c7
:103500000482d2008582d2000000a0000202520094
:1035100083825a0003003b000202420083824a0079
:103520000000a1000603e900f3ff3a0000000600d6
:10353000810378003f0207000001be006000b80070
:103540000478a30013003a006220e10015003e0059
:103550000d0039008301d1000281d3008180d300a6
:103560008301d1000281d3008180d3008301d10087
:103570000281d3008180d3000538b000c42add0069
:10358000f300b2008381720007f0a70003f0a000ef
:1035900000000600f3ff2700f2ff2f006110b900c2
:1035a000fbff370003ff2700f7ff3700881f780075
:1035b000000478005001be004000be00040040003e
:1035c000858048000601490087814900009cbe00b3
:1035d0000294be000400e1000588e1000690e100cd
:1035e0000798e10002003100680044001008e8007c
:1035f0004f047800000006001000fa00889fbe000b
:103600008a9fbe003004be002005be00c8b79f00e0
:10361000d9b79f00eab79f00fbb79f00040454008e
:1036200085845c0006055d0087855d0088bf9f007e
:1036300099bf9f00aabf9f00bbbf9f000898be0014
:103640000a98be008000eb004fb49700dfb49700eb
:103650006fb59700ffb597000440e10005c8e10091
:1036600006d0e10007d8e100010031001100200080
:10367000108810004f05be004f04be000080fa0005
:10368000000006001200fa00889fbe008a9fbe005c
:103690008c1f78000205be000004be00f4b79f0036
:1036a00085bf9f0096bf9f00a7bf9f000000eb0053
:1036b000e0b79f00d0b79f00c0b79f00b0b79f0092
:1036c000a0b79f0000067800dfb097006fb09700aa
:1036d000000140000000e0000a003d008c000700ef
:1036e00001003d00120020009200070001003d0093
:1036f00012002000970007007c805700abff0700f6
:10370000090037008200070001003d001200200080
:103710008800070001003d00120020008d00070016
:103720007c805700b4ff07006fb297000400e000f0
:103730000700350010002000010020006011b800d3
:1037400008047000898470000a0571008b8571007f
:103750000c06e800f0032000800f5600daff34006a
:103760000400e00006003d007fb297008fba97008a
:103770001fbb9700afbb97007c8057008bff0700f3
:103780006fa897000000e00004003a002fb49700f3
:10379000bfb497004fb59700dfb5970089000700c9
:1037a0004f0678004f05be004f04be000080fa00af
:1037b00000000600881f780018002000881f78008d
:1037c000b0ff07008f87e9004f0478000000060073
:1037d000801feb00abff07008f87e90000000600a9
:1037e000889fbe008a9fbe008c1f78006e00070075
:1037f00005003d002f00070007003d003d000700c9
:103800000006eb00040037003f00070002003d0007
:10381000300007001c0020006a000700e5ff0700d9
:103820000203be000002be000c00e00001003200f6
:10383000280007000400be000601be004f06780005
:103840004f05be004f04be0000000600889fbe006a
:103850008a9fbe008c1f78005300070003003d00c4
:103860001400070006003d00040037002600070092
:1038700003003d006000b8006011b8001d000700a3
:1038800050000700d2ff07000203be000002be0086
:103890000c00e000010032000e0007000400be0032
:1038a0000601be004f0678004f05be004f04be0063
:1038b000000006006000b8006011b8000804500065
:1038c000898458000a0559008b8559001c00200086
:1038d000030037006000b8006011b8000500370031
:1038e000e00f5200e08f5a00e00f5b00e08f5b00ba
:1038f00000000600040250008582580006035900ab
:1039000087835900000006000006eb00f4ff370033
:103910004f08de0000007100c0b79f00018040002a
:10392000b0b79f000001eb00afb097000100e000ce
:103930000000060002007000b0b79f000180400048
:10394000a0b79f000001eb009fb097000100e000ce
:103950000000060002007000a0b79f000180400038
:103960000fb29700cf20de000100700090b79f00db
:1039700004024200130007004f18de00000272002c
:1039800084b79f000804440089844c000a054d0058
:103990008b854d005fb29700efb297007fb3970021
:1039a0008fbb9700000006000205be000004be00a9
:1039b000e00f5000e08f5800e00f5900e08f5900f1
:1039c000000006000800be000a01be00000006005c
:1039d0008f1fd1002c0107008f87e9000000e00055
:1039e000000006001400fa00889fbe008a9fbe00f7
:1039f0008c9fbe000004be000205be0068004700a8
:103a00000a90be000890be00480107000070a700a1
:103a10000bf0a100304320009e02900080825200f3
:103a2000b0fe2f000028e10011003d00b0fc2f0087
:103a30000028e100150034001e0990008e08900057
:103a40007e0090000501b0000201d1008180d3000a
:103a50000080d3008502e800fbff3a000b00e00085
:103a60006d013b0060001000e08018006a01370023
:103a7000f0ff2f00f1ff27000b00e00066013b0084
:103a80000100280000002000630137006000b8003a
:103a9000610137004f89de00820178006301370041
:103aa00007f0a20098013700809feb00f6000700a6
:103ab0008f87e9000000e00000000600839f680097
:103ac0000100e00002003d0060001000e0801800ee
:103ad0000300e00002003d0060011100e0811900d8
:103ae00083fe07004f00e00002003b006000100072
:103af000e0801800000006002800fa00889fbe0041
:103b00008a9fbe008c9fbe0003866b002e010700bb
:103b10000028a30064003a000128a30067003a00cf
:103b20000008a30062003a000108a30065003a0003
:103b30001e009000be08900081064000ed3fb100dd
:103b4000f4805700ee019000111ab8008e09900021
:103b5000311bb8009e099000311cb800511db800ff
:103b6000f485570046000700fe0190003a00070068
:103b70008b85e8003e0007008e099000400007009a
:103b8000ee019000340007008b85e8003800070044
:103b90008e099000400007009e0990001b18b80095
:103ba000890440000a854800fe01900034000700a7
:103bb0008b85e80038000700ee0190003000070018
:103bc0008e0990001b18b800890440000a8548003f
:103bd0000a98a30008003a000402420085824a00c5
:103be00006034b0087834b0008044c0089844c007b
:103bf0000a054d008d06e90084827200850273007b
:103c00004c3add00850272000100320015002000f0
:103c1000443ade001400b2004538de00cb45dd003a
:103c20000b007000c540de00cb4ddd008b807000c6
:103c30004549de00cb55dd000b017100c551de00aa
:103c40000d037800ad01070003f0a1000cf0a70000
:103c500003f0a000f00037001b18b80085024000f8
:103c600006834800e0834b0060044c0007003700e7
:103c70001b18b8000603400087834800faff37008e
:103c80001b18b8008703400008844800e0844c00fb
:103c900060054d00000006001b18b8000804400035
:103ca00089844800faff37000108a300d7003a00d2
:103cb0005800be005801be00e3ff37000008a30013
:103cc000d2003a0009047800f9ff37002800fa0012
:103cd000889fbe008a9fbe008c9fbe0003866b003b
:103ce000b90007006400e100440032006408e1000c
:103cf0004a0032006100e100460032006108e10044
:103d000049003200ec0647006000b8003d02be00ea
:103d10003d03be00f48657006011b8003d04be00ac
:103d20003d05be007d0320000b0037000000a00011
:103d30008d06e900130032000402420085824a0029
:103d400006034b0087834b00000040008180480041
:103d500002014900838149000802520089825a0009
:103d60000a035b008b835b00f0ff3b00080242000c
:103d700089824a000a034b008b834b008d06e900c1
:103d8000edff3a008482720086827200f707b2006b
:103d90008782720001003200150020001e0490008e
:103da0003e0b900006035400e63fb0000368a300fa
:103db000070032000000a7000500a0008301d10029
:103dc0000281d3008180d3000080d3000603e80085
:103dd0008301d1000281d3008180d3000080d30011
:103de0000002eb000482d2004401070003f0a100ae
:103df0000cf0a70003f0a000870037006402470022
:103e00006408e100810032003400be003401be00cd
:103e1000f6ff37006108e1007c0032006011b80055
:103e20006000b800f1ff370003ff27000200200008
:103e3000fbff3700c70ade00f107b200f50fb20042
:103e400008003200e1cf4200020032000170a00001
:103e500024000500810f70000100320004080500f5
:103e600044000500810f700002003a0014000500b4
:103e70008502e9000000400081c04800fcff3b00d3
:103e80000170a00024000500889fbe008a9fbe002c
:103e90008c9fbe000404be000605be00809fbe00cd
:103ea000829fbe0041010700040678000800be00a2
:103eb0000a01be003d010700840678004f03be00e2
:103ec0004f02be008d4f76007fb097001300330085
:103ed000f0ff2f008b8f6b0006003b000d06660085
:103ee0000c00a7000a00370007f0a6001000200011
:103ef0000a003700880f5200898f5a008a0f5b0032
:103f00008b8f5b00030039001000200001003e0091
:103f10000000200007f0a7000000ea004f06be00e6
:103f20004f05be004f04be00000006008000780070
:103f30005002be005003be004439de00f700b2005c
:103f4000f37f200003016100090032000218e10044
:103f500016003a00850172008301730083817300ab
:103f60000008200015003a00400020001300370030
:103f700085017200830173008381730005003a009c
:103f800004a8be0006a8be00100020000b003700e9
:103f90000201e9000402420085824a0006034b0048
:103fa00087834b000748a300f9ff32000740a000b9
:103fb00004a8be0006a8be002000200080009800d3
:103fc0009200980000000600680447000294be00ba
:103fd0000094be00fc0447008694be008494be009a
:103fe00009007800d1ff070008007800cfff070024
:103ff00099007800814f70000b003b000800be0064
:10400000fc0007004f00b10003003700f3ff27005a
:10401000f2ff2f006110b9004f06be004f05be0031
:104020004f04be000080fa0000000600889fbe001a
:10403000830478000300e0002c00350003003c00fe
:104040000082700004027100260032003643200016
:10405000c50020008383cf000a0039000541b1006c
:104060008283cf00070039000541b1008183cf0072
:10407000040039000541b1008083cf000100390000
:104080000541b10085c353006022b8001200320020
:104090000a003b0084827200610260008301d1004b
:1040a0000281d3008180d3000080d3000603e800a2
:1040b0008743e800f7ff3a000700370000004000a0
:1040c0008180480002014900838149000603e9001c
:1040d0008743e900f9ff3a008800070009f0a700cc
:1040e00003f0a0004f04be000000060060001000b6
:1040f000e080180060011900e0811900d3ff3b0047
:10410000033e2c00f7ff37002800fa00889fbe000e
:104110008a9fbe008c9fbe000706780087866900d4
:104120000c003b00030478008704780008f0a1002d
:1041300009f0a100840f5000858f5800860f5900a8
:10414000890f5c00030033000cf0a20001003a006c
:104150000cf0a1009cff07006400e1005f0032004a
:10416000780147006408e100610032006c014700fb
:10417000748557003200be001201be003a04be0032
:104180001a05be001e039000be0a9000850353006e
:1041900006003d000004fd008104fd000205fd0055
:1041a0008305fd008703ea00050378000df8a300ee
:1041b0000400320060041400e0841c0060051d004f
:1041c000e0851d006022b8007d0320000d38e1006d
:1041d0008006eb000b0039004433dd00f300b20031
:1041e0008301730039003700848272000d02780069
:1041f000e10664008b85d1000a85d3008984d30051
:104200000884d3008703e900f7ff3b000800400063
:10421000898048000a0149008b81490004003b0065
:1042200060001000e080180060011900e0811900b2
:104230000358a300090032008d827200848272004c
:10424000610260008301d1000281d3008180d3002c
:104250000080d3000603e8001b0037000348a300da
:1042600017003a000600e000170034000603e900da
:104270000d00a300000048008180480002014900b1
:10428000838149000348a3000f003a000600e000c4
:10429000090034000603e900000040008180480066
:1042a000020149008381490001003a000003eb004c
:1042b0000348a300f5ff32006022b8000200370077
:1042c00084827200618266000c00070003f0a10086
:1042d0000cf0a70003f0a0004fff37006401470077
:1042e0006408e10002003a000df8a30047ff3a001d
:1042f0003200be001201be0047ff37001800200048
:1043000057002000080453000d003d000600200067
:1043100097fc2f000740e1001e00340084827200e9
:10432000610260008301d1000281d3008180d3004b
:104330000080d3000804e800f8ff3a00470020009e
:104340006104600005047400040464000d00320080
:1043500061004000e080480060014900e0814900c0
:1043600003b8a500070032000603e8006538e10045
:1043700004003a008301d1000281d3008180d30080
:104380000080d300f87f20000830e10003003500f2
:10439000080378006000b8006011b8004433dd0005
:1043a000f300b200830173000000060005ff270040
:1043b00005826100070032000428e100010032009c
:1043c000240005000600070001003a004400050033
:1043d0000408050002000700f9ff3a001400050078
:1043e0006f82610081027000850271008502720097
:1043f00000000600e48240001078a30007003200ad
:10440000640240001178a3003400be001401be0015
:10441000040032000330a700000006003500be0093
:104420001501be000330a00000000600000888004f
:10443000000006008c60a90005e1a9008460a900c5
:1044400000000600901c8800a11c880000000600e7
:10445000401bde0007002000e1cf520003003200c5
:10446000e2cf52000500320008003700801a8800b1
:10447000961a8800a21a880007003700001a8800e0
:10448000161a8800221a880003003700001b8800d3
:10449000161b8800221b88000001eb000a00370071
:1044a00060352000e1cf5200040032006036200069
:1044b000e2cf520001003a00603420001170790010
:1044c0000201e8008100e8000480fb00800f510039
:1044d000f3ff3500e1cf52000d003200e2cf520071
:1044e000160032006f4062004300dd0041362000bc
:1044f0009140780072c8b30082c0600080c0700034
:104500000100780064e3b7006e63a80000000600b5
:104510006f4062004300dd0041352000914078008b
:1045200072c8b30082c0600080c0700001007800d3
:1045300054e3b7005e63a800000006006f4062000d
:104540004300dd00413420009140780072c8b30080
:1045500082c0600080c070000100780044e3b700b2
:104560004e63a800000006000004e00004003200d2
:104570008000eb00e14f500006003a0002003700d7
:104580008ec3bf00010037007ec3bf000080fb0068
:10459000c700de0001007800000006000002eb000a
:1045a00080017800090037000204e00003003200b7
:1045b00060372000e14f51000100320060382000d8
:1045c000e0497a000402e8008301e8000180fb0072
:1045d000800f5200f4ff35000000060080007800d4
:1045e000000178000cc2bf0066406000e64f50003a
:1045f00010003a00050037000fc2bf000018a300ea
:10460000fdff3a00821088008180e80011017800e7
:104610000200e000f8ff3a00000006000fc2bf00f1
:104620000018a300fdff3a000100fb008010880085
:104630000201e800924078000104e000f7ff3a0030
:1046400000000600a2108800601088007110880029
:10465000000006008520a9008540a900e741600010
:10466000c419dd008109200091407800f2c8b30030
:1046700082c0600083c070008000fd0098e0b70039
:104680008000fd00800178000307b200c419de003d
:10469000910920009140780082cfb30082c0600071
:1046a00083c070008000fd0099e0b7008000fd002d
:1046b000680160004311de0002414100d108200082
:1046c000914078000114a10082c070008000fd00bc
:1046d0008de0b7008000fd000008b2004700de005a
:1046e0004200dd00d1082000914078000124a100a3
:1046f00080c07000010078008de0b7000000060067
:10470000801c880000000600e14f500003003200ca
:10471000e24f50000300320004003700f11a880015
:1047200000000600711a880000000600711b880056
:10473000000006000004e00004003200e14f5000d9
:1047400002003a00f11b880000000600711c88007e
:10475000000006009623ef008760a900c01c8800b7
:10476000e7c16000c419dd00a1c0bf00f2c8b300fa
:104770000240600003407000a1e0b700e8806000e4
:10478000c308de00c308dd008fc0bf000034a100f5
:10479000014070008fe0b700000006000021ef002c
:1047a0001108880020088800000006008460a90025
:1047b000e7416000c419dd005109200091407800f4
:1047c000f2c8b30082c0600083c070008000fd00aa
:1047d00095e0b7008000fd00680060004300de0047
:1047e0004300dd00c1082000914078000134a100a1
:1047f00080c07000010078008ce0b7000000060067
:104800000cc2bf0066406000e64f500002003a0054
:10481000901080000000060090108000f00fb200a1
:104820000000060097c3bf004500de006100600085
:10483000000006009bc3bf000080fb0000000600d4
:104840009ac3bf000080fb000000060097c3bf00b2
:104850004300de00610060000000060097c3bf0057
:104860004400de0061006000000006003600f80031
:10487000809fbe00829fbe00849fbe00869fbe00b8
:104880003400f80000c0b300a00188000000fa0066
:104890000000eb00e5fe0700f7cbbf000040e8009a
:1048a000f7ebb700f7cbbf00e84f5000050036002c
:1048b0000040eb00f7ebb700defe070010c0b300ce
:1048c000f6ebb7008460a9000080fa003400f9001c
:1048d0004f03be004f02be004f01be004f00be009e
:1048e0003600f900004006003600f800809fbe0048
:1048f000829fbe00849fbe00869fbe003400f800e9
:1049000000c0b300a00188001000fa006000b800e9
:1049100020079800310798006000b800008fbe00a3
:104920006000b8006011b800400798005107980077
:1049300062079800730798008760a90090c3bf00c2
:104940006e406000e24f50000a003a0097c3bf007b
:1049500001c8b300014060000004e0000200320022
:1049600010c0b300f4ebb70097e3a90096a3a90029
:10497000ab0037009603a90084c3bf006f406000fe
:104980000080fb006f0160001155800000ff2f00c8
:104990000080600002007000105588008ec3bf00c8
:1049a000684060000004e0003b00320080c3bf00ac
:1049b000614060000004e0002d003200a28aa800df
:1049c000a2aaa800101c800001002000f05488005a
:1049d0000155880085c3bf000080fb004200de0057
:1049e0000080fb0001002000008fbe00001c800042
:1049f0004200de00f17f2000010060000100200085
:104a00002007980031079800f0548000015580007d
:104a10004609dd00ca00de00810071004600dd00ad
:104a2000f0548800015588002e009000be009000d0
:104a3000c200dd0000002000200798003107980028
:104a4000f2548000035580002e009000be009000bc
:104a500000007100818071003e017000ae81700025
:104a60000200be00f0548800015588005300370052
:104a7000a28aa900a2aaa800001c80004200de00b1
:104a8000f17f20000100600001002000f054880048
:104a9000015588004900370080c3bf0061406000b5
:104aa0000004e0002d003200a28aa800a2aaa900fa
:104ab000101c800001002000f0548800015588007f
:104ac00085c3bf000080fb004200de000080fb00c9
:104ad00001002000008fbe00001c80004200de00ac
:104ae000f17f2000010060000100200020079800f5
:104af00031079800f054800001558000c609dd00a0
:104b0000ca00de00818071004600dd00f05488009c
:104b1000015588002e009000be009000c200dd000c
:104b2000000020002007980031079800f254800010
:104b3000035580002e009000be0090000000710020
:104b4000818071003e017000ae8170000200be00e5
:104b5000f05488000155880009003700a28aa90096
:104b6000a2aaa900001c80004200de00f17f200004
:104b70000100600001002000f05488000155880009
:104b800084c3bf006f40600080407800c0b1200047
:104b900015030700e8004700c0b12000200307000c
:104ba0004e009000de0090006e019000fe0190002b
:104bb00044aa2000009abe000292be00b9cbbf00fa
:104bc0000004e00014003400b7cbbf000080fb00fd
:104bd0006e00b90080007800c0aa2000008040006c
:104be000e1a9200043030700b7cbbf000040e80065
:104bf000b7ebb700b7cbbf00e84f500002003a0058
:104c00000040eb00b7ebb700b9cbbf000040e900b4
:104c1000b9ebb7000200370010c0b300f5ebb700e6
:104c20008ee3a9000080fa003400f9004f03be00b3
:104c30004f02be004f01be004f00be003600f9001b
:104c4000004006000200fa00004f780011392000f1
:104c50009140780080cfb30000c060000024a00025
:104c600091e3b70090c3bf000080fb004500de0069
:104c70000080fb00e30f5000faff34001e80fb00b1
:104c800001eb2b004300dd000080e800608078002d
:104c90000000e900e7006000807f240000817000d0
:104ca0001e80fb0001eb2b004300dd006400400090
:104cb000608078000000e90067006000c300dd004c
:104cc000707c240000807000000161001e80fb00e9
:104cd00001eb2b004300dd0066004000608078009f
:104ce0000000e90067006000c800dd00f00f24004c
:104cf0000080700080006100f07f20000081600073
:104d00001e80fb0001eb2b004300dd00e0807800fb
:104d1000000420000080700082007800c9fd0700b8
:104d2000113920009140780080cfb30000c06000ae
:104d300091e3b70090c3bf0001ceb3000140600013
:104d40000004e000fbff3a000080fa0000000600cb
:104d50001200fa00008fbe00424798001e00be00fd
:104d6000805f8800915f88001139200091407800b1
:104d700080cfb30000c060000024a00091e3b70022
:104d800090c3bf000080fb004500de000080fb00f8
:104d9000e30f5000faff34003003a8004e409000ab
:104da000e14f50006c003a000803a800000020000a
:104db000c1ff21009e0178001e02900000017800d2
:104dc0000100780002816100000062006102b80009
:104dd00034079800450798003e029000ce029000ec
:104de000c020dd00000020006112b80034079800e8
:104df000450798003e019000ce019000020070002f
:104e000083807000008fbe001e00be004208de00de
:104e100001002000008fbe009e007800f07f20007f
:104e200080806000f07f2000008060004201dd0093
:104e30008119800030002e000080600002007000a8
:104e400080198800845f8000955f8000048fbe0019
:104e500000fc2f00310020009e0178001e0290000f
:104e6000000178000100780002816100000062000a
:104e70006102b80054079800650798005e02900030
:104e8000ee029000c020dd00000020006112b8009a
:104e900054079800650798005e019000ee019000ad
:104ea0000200700083807000008fbe001e00be00f4
:104eb000ca09dd004600de0000807100c608de0081
:104ec000008fbe001e00780090198800845f80006b
:104ed000955f8000048fbe00f003200001002000d9
:104ee0009e0178001e029000000178000100780009
:104ef00002816100000062006102b800740798003e
:104f0000050f98007e0290008e0a9000c020dd0000
:104f1000000020006112b80074079800050f980087
:104f20007e0190008e099000020070008380700066
:104f3000008fbe001e00be00ca09dd00c600de00f4
:104f4000818071004a00dd00008fbe001e007800e5
:104f5000a0198800140037000803a9009e007800fb
:104f6000f07f200080806000f07f200000806000e3
:104f7000f17f200001006000f17f2000010060004f
:104f80004201dd008119800030002e0000806000a9
:104f900002007000801988000000eb009019880062
:104fa0000000eb00a0198800801980004200de009c
:104fb000f17f200001006000405f8800113920006f
:104fc0009140780080cfb30000c0600091e3b7004b
:104fd00090c3bf0001ceb300014060000004e000b8
:104fe000fbff3a000080fa00000006001200fa0001
:104ff000008fbe00424798001e00be00605f880020
:10500000715f8800113920009140780080cfb30093
:1050100000c060000024a00091e3b70090c3bf006f
:105020000080fb004500de000080fb00e30f500025
:10503000faff34003003a8004e409000e14f5000ca
:105040007d003a000803a80000002000c1ff2100f5
:105050009e0178001e029000000178000100780097
:1050600002816100000062006102b800340798000c
:10507000450798003e029000ce029000c020dd005f
:10508000000020006112b80034079800450798001e
:105090003e019000ce0190000200700083807000fd
:1050a000008fbe001e00be004208de00010020008e
:1050b000008fbe009e007800f07f2000808060009e
:1050c000f07f2000008060004201dd0001188000b8
:1050d00030002e0000806000020070000018880080
:1050e0000003a8009e007800f07f20008080600010
:1050f000f07f2000008060004201dd004118800048
:1051000030002e000080600002007000401888000f
:105110000803a800645f8000755f8000048fbe00f4
:1051200000fc2f00310020009e0178001e0290003c
:105130000001780001007800028161000000620037
:105140006102b80054079800650798005e0290005d
:10515000ee029000c020dd00000020006112b800c7
:1051600054079800650798005e019000ee019000da
:105170000200700083807000008fbe001e00be0021
:10518000ca09dd004600de0000807100c608de00ae
:10519000008fbe001e007800101888001e007800e6
:1051a00050188800645f8000755f8000048fbe0027
:1051b000f0032000010020009e0178001e029000f4
:1051c00000017800010078000281610000006200a7
:1051d0006102b80074079800050f98007e029000e5
:1051e0008e0a9000c020dd00000020006112b8008f
:1051f00074079800050f98007e0190008e099000ba
:105200000200700083807000008fbe001e00be0090
:10521000ca09dd00c600de00818071004a00dd00a1
:10522000008fbe001e007800201888001e00780045
:1052300060188800280037000803a9000003a900af
:105240009e007800f07f200080806000f07f2000ca
:1052500000806000f17f200001006000f17f2000ed
:10526000010060004201dd000118800030002e00c6
:105270000080600002007000001888000000eb0051
:10528000101888000000eb00201888009e007800ad
:10529000f07f200080806000f07f200000806000b0
:1052a000f17f200001006000f17f2000010060001c
:1052b0004201dd004118800030002e0000806000b7
:1052c00002007000401888000000eb0050188800b1
:1052d0000000eb0060188800001880004200de002b
:1052e000f17f200001006000505f8800113920002c
:1052f0009140780080cfb30000c0600091e3b70018
:1053000090c3bf0001ceb300014060000004e00084
:10531000fbff3a000080fa00000006003e00fa00a1
:10532000605f980002179800131798004167980073
:10533000546798000040eb0040579800f00f2000a1
:10534000010020006011b800500798006107980024
:1053500072079800030f98000040eb002057980058
:105360001d0037002e5090000081fb001eb89700f2
:10537000804078005e00900080c0600075004700ab
:10538000017178001eb89700aeb897003eb997003b
:10539000ceb997004800de00480add000000720028
:1053a000c808de004812dd00810072004811de00ee
:1053b000481add0002017200c899de0010bf9f008c
:1053c00021bf9f0032bf9f0043bf9f002e5090001f
:1053d0000040e800205798002e509000e74f500002
:1053e000e0ff36006e589000e14f50004a003a004e
:1053f0004e609000e14f500009003a00f08f2f00fe
:105400001007980080ff2f00f10f2f002007980051
:1054100031079800f08f2f00000f78000800370048
:10542000f08f2f001007980080df2f00f10f2f0062
:105430002007980031079800d08f2f00000f7800c8
:105440000e1090009e10900002002000c3ff21006b
:105450000002780081027800020078008300780062
:1054600000016200018062006102b80034179800f8
:10547000451798003e129000ce129000c020dd002b
:10548000000020006112b8003417980045179800fa
:105490003e119000ce1190000200700083807000d9
:1054a0004208de0001002000400798000e10900026
:1054b0009e109000f2ff2f003300200000027800c1
:1054c0008102780002007800830078000001620009
:1054d000018062006102b8005417980065179800b7
:1054e0005e129000ee129000c020dd00000020004f
:1054f0006112b80054179800651798005e1190006b
:10550000ee11900002007000838070000017980078
:1055100011179800190037004e609000e14f5000bd
:1055200009003a00e08f2f0010079800f08f2f003d
:10553000000f780080ff2f00f10f2f002007980048
:105540003107980008003700e08f2f0010079800ff
:10555000d08f2f00000f780080df2f00f10f2f0079
:1055600020079800310798008e119000430798009b
:105570006000b80000179800111798000e109000f6
:105580009e10900002002c003300200000027800e2
:105590008102780002007800830078000001620038
:1055a000018062006102b80074179800051f98001e
:1055b0007e1290008e1a9000c020dd0000002000b6
:1055c0006112b80074179800051f98007e119000b2
:1055d0008e19900002007000838070004e0bdd0079
:1055e000c203de00870373004e03dd000e1090003f
:1055f0009e10900002fc23000300200000027800af
:1056000081027800020078008300780000016200c7
:10561000018062006102b800141f9800251f9800e5
:105620001e1a9000ae1a9000c020dd00000020007d
:105630006112b800141f9800251f98001e199000d1
:10564000ae1990000200700083807000ca09dd006e
:10565000c600de00818071004a00dd000003730097
:10566000818373000e1090009e109000f2032000c2
:105670000300200000027800810278000200780018
:105680008300780000016200018062006102b800be
:10569000341f9800451f98003e1a9000ce1a9000c3
:1056a000c020dd00000020006112b800341f980007
:1056b000451f98003e199000ce199000020070001e
:1056c00083807000ca09dd00c600de0081807100a1
:1056d0004a00dd000001730081817300803f2000db
:1056e0000100200000007100818071002e019000f7
:1056f000be0190000002780081027800020078006c
:105700008300780000026200018062006101b8003d
:10571000521f9800631f98005e189000ee189000ca
:10572000c001dd00020020006120b800501f980079
:10573000611f98005e1a9000ee1a9000040171003b
:1057400085817100ce009000007c20000080600008
:105750004502dd00ce009000f003200000806000d4
:105760004200dd0000007200800078003100b300cc
:105770001e009000008060001e006000f5004700e1
:10578000ce5290005e62900031fb07007901070065
:105790006ec3bf00684060000004e00003003200f8
:1057a000f6cbbf00e14f5000f9ff3a00f6cbbf0047
:1057b000e14f500003003a000040eb00f8ebb70067
:1057c0000200370010c0b300f8ebb7000000eb0098
:1057d00016fb07000040eb00f7ebb70015fb0700d6
:1057e0000080fa00000006000400fa00000f7800b4
:1057f000214798000040eb005bfb07000004e0003d
:10580000fcff32000041eb00ae4090001e0078002b
:1058100062fb07008ee3a9000080fa00000006008a
:105820001000fa0060079800710798006000b80047
:105830006011b800200798003107980042079800cf
:1058400053079800640f47000040eb002047980082
:105850000d0037002e4090000000fb008000780013
:105860006e0090000080400010407800804078007a
:105870001e007800014878002e4090000040e800ab
:10588000204798001e0fe8002e4090008000fb008b
:10589000105580006f4060000080fb00808f50003a
:1058a000ecff3500070037009e0078000040eb0059
:1058b000804878001e0fe8002e4090000040e8006d
:1058c000204798002e409000e74f5000f6ff34002c
:1058d0002e009000be0090004e019000de0190006e
:1058e0007e029000009abe000292be000080fa0084
:1058f000000006000400fa00000f7800110798006d
:105900009e0078001e00900006000900b018780084
:10591000e100b100e000b1000080fa0000000600e4
:105920003000fa00881f7800b8cbbf000080fb0071
:105930006e00b900e4004000c0aa200000804000d2
:10594000100078004400de0061406000e14f50002c
:1059500003003a0080c5b3002047980002003700da
:1059600030c5b30020479800b8cbbf000080fb00d3
:105970006e00b900e4004000c0aa20000080400092
:10598000100078004500de0061406000e14f5000eb
:1059900014003a0020c5b300104798001e40900044
:1059a0008081fb00b8cbbf000080fb006e00b90017
:1059b00080007800c0aa2000008040001000be00d7
:1059c00063014700831f7800809fbe0080d12b00b9
:1059d000801f7800020078007bea0700e887570004
:1059e00027003700e0c4b30010479800b8cbbf00d1
:1059f0000080fb006e00b900e6004000c0aa200055
:105a0000008040003002be002003be00b8cbbf00c3
:105a10000080fb006e00b900e4004000c0aa200036
:105a200000804000100078006f4060008081fb0023
:105a30001e4090000084fb00b8cbbf000080fb003c
:105a40006e00b90080007800c0aa200000804000ed
:105a50001000be0063014700849fbe00869fbe0009
:105a6000831f7800881f7800809fbe0030d22b00f3
:105a7000801f78000200780053ea0700f287570081
:105a800063004700d5fa0700b8cbbf000040e8002c
:105a9000b8ebb700b8cbbf00e84f500002003a00a7
:105aa0000040eb00b8ebb7008f60a9009803a90095
:105ab000b9cbbf000040e800b9ebb7008f60a80089
:105ac0009803a8008760a9009603a9004f047800f6
:105ad0000080fa00000006000000fa00f4cbbf00ce
:105ae000e14f500006003a008f60a9000040eb0033
:105af000f4ebb7008f60a80080d32b00b7fa070043
:105b0000f5cbbf00e14f500006003a008f60a900be
:105b10000040eb00f5ebb7008f60a800f0d72b003a
:105b2000aefa0700f6cbbf00e14f50000a003a0082
:105b30008c60a9000040eb00f6ebb7008c60a80079
:105b4000a0db2b00a5fa070010df2b00a3fa07004b
:105b5000a0e32b00a1fa07000080fa000000060075
:105b60000000fa00dcff0700b9cbbf00e74f500090
:105b700001003c006aff07000080fa0000000600f8
:105b80000000fa000080eb00501688000080eb0057
:105b9000301688000080eb00401588000000eb0004
:105ba000801688000080eb00601688000000eb0083
:105bb000b01688000080eb00901688000000eb0013
:105bc000e01688000000eb00c01688000000eb0023
:105bd000101788000080eb00f01688000080fa00a3
:105be000000006000000fa009f000700f2002000fd
:105bf000f1772f0000f02d0092fa07000080fa00e4
:105c0000000006000000fa00e0f72f0091fa0700fc
:105c10000080fa00000006001000fa00200798003b
:105c200032079800430798005407980065079800ca
:105c3000614f980000c02000b1fa070090c3bf0078
:105c40000080fb004500de000080fb00e30f5000f9
:105c5000faff34002e00900001eb2b004300dd0022
:105c60000080e800608078000000e900e700600044
:105c7000807f2400008170002e00900001eb2b003b
:105c80004300dd0064004000608078000000e9000f
:105c900067006000c300dd00707c2400008070009d
:105ca000000161002e00900001eb2b004300dd009d
:105cb00066004000608078000000e9006700600036
:105cc000c800dd00f00f240000807000800061003b
:105cd000f07f2000008160002e00900001eb2b007f
:105ce0004300dd00e08078000004200000807000a8
:105cf00082007800d3f907006e4990005e009000a2
:105d0000ee009000b9fc07006e4990003e00900044
:105d1000ce0090000efc07000000eb00000f7800a2
:105d20001e0078003100200077fa07001e0078007e
:105d30008000eb007ffa07000080200070fa070067
:105d400090c3bf0001ceb300014060000004e0003a
:105d5000fbff3a000080fa00000006000000fa0095
:105d6000d1ff2f00100220007afa07000080fa000d
:105d7000000006000000fa008080eb0090fb2d0080
:105d800086fa0700c0ff2f0088fa07000080fa009b
:105d9000000006000000fa0079ff070011c0b30000
:105da0006022b8006011b8000000eb009aff070005
:105db000eaff07008bff070092ff070080ee2b0031
:105dc00055e90700d0f22b0053e9070020f72b001c
:105dd00051e90700e801070061ff0700fdff3700f8
:105de0003600f800809fbe00829fbe00849fbe00e8
:105df000869fbe003400f80000c0b300a0018800f8
:105e00000200fa008520a9007dfa0700004f780003
:105e10009e407800e0902000cf0607000004e000dc
:105e200002003a00a0fb2b00ecf907000ec2bf00f5
:105e3000624060000004e000030032000e22a9006e
:105e400050ff2b00e5f907000080fa003400f9004c
:105e50004f03be004f02be004f01be004f00be0008
:105e60003600f900004006000000fa00f20f2000a2
:105e700061912000e09020002d060700e0902000b6
:105e8000e40607000080fa00000006000800fa009f
:105e9000881f78000000370042c0bf000080fb0070
:105ea0004500de00404798009002800010079800ef
:105eb000ff3ffc00210420009140780000ceb30099
:105ec00000c0700042e0b7001e0090009002880001
:105ed000e09020002806070070479800900280009c
:105ee000000f7800ff3ffc004e40900067406000cc
:105ef000c500dd0042c0bf007f406000014070006f
:105f000042e0b7001e007800900288007e409000ba
:105f10000004e00047003200fdcbbf000084fb001e
:105f20007e4090000000fb0008e9070080407800f8
:105f3000e0bf200000004400014878007e4090004f
:105f4000ed4f500005003200d1bf20009140780095
:105f5000c0c2b30080cf500028003a00fdcbbf0084
:105f60008080fb00e0bf2000808040000040eb000c
:105f700080487800e0bf2000870107006047980054
:105f80006e4090000004e00019003a00fccbbf0016
:105f90000004e00014003400facbbf000080fb00d6
:105fa0007e00b90080007800e08120000080400081
:105fb0000180200022000700facbbf000040e8006b
:105fc000faebb700facbbf00e84f500002003a00ee
:105fd0000040eb00faebb700fccbbf000040e9004b
:105fe000fcebb7000200370000032c007bf9070030
:105ff0000040eb00fdebb700a7ff37007e409000ac
:10600000e84f500007003a00fdcbbf000004e0005d
:1060100004003200fdcbbf000040e900fdebb700fb
:106020009dff3700fdcbbf000040e800fdebb7004f
:1060300099ff37004f0478000080fa000000060046
:106040000400fa00000f7800110798009e00780005
:106050001e0090000e000900b0187800e101b100a8
:10606000e001b1009e0090000040eb00e048980085
:106070001e0190006000b8000089be001e02900062
:106080006000b8006011b80030029800410298002a
:1060900052029800630298009e0090002100900038
:1060a0000000a1000010a1000020a1000030a1000c
:1060b000a00098009e009000210090000040a100e8
:1060c000a00098009e009000210090000050a100c8
:1060d000a00098009e009000210090000060a100a8
:1060e0000070a100a00098000080fa0000000600e7
:1060f0000600fa00000f78001207980023079800a6
:10610000d0062c0035f907009e007800a0e72b0090
:1061100095e807000000e00003003a001e00900030
:10612000c8fa0700270037009e00780030e82b00ef
:106130008de807000000e00006003a0062bb200086
:10614000124178001e009000ae00900000fb070096
:106150001c0037009e007800c0e82b0082e8070092
:106160000000e00006003a0062bb20001241780007
:106170001e009000ae0090009cfb0700110037004d
:106180009e00780070ea2b0077e807000000e0002e
:106190000c003a001e009000b6ebb70062bb200076
:1061a00012417800605f8000715f80008ffb070004
:1061b00062bb200012417800805f8000915f800008
:1061c000e3fa07000080fa00000006004400fa002d
:1061d000002798006000b8005007980061079800f9
:1061e0006000b80030079800410798006000b800d0
:1061f00010079800210798000040eb00004f78003e
:10620000060037009e00fb006e00470080804000c3
:106210000040eb00804878001e4fe80010c3b30038
:106220009e4f1000f7ff34008e209000a0e72b0057
:106230004de807000000e00035003a0092c3bf00bf
:10624000f043b2000080fb00102798001e20900051
:10625000e70f5000220032009e209000e78f500090
:106260000a003c001e209000e20f50001600320091
:106270009e209000e58f5000160032001e209000f6
:106280000000e0000d003200820037001002200004
:106290009e209000808f500017003200a003200045
:1062a0009e209000808f5000160032001e2090002b
:1062b000fc0f50000d0032007600370000072c0064
:1062c000c6f807007300370090082c00c3f80700d9
:1062d00070003700500a2c00c0f807006d0037002e
:1062e000100c2c00bdf807006a003700d00d2c0000
:1062f000baf8070067003700800f2c00b7f80700d6
:106300006400370030112c00b4f80700610037003a
:106310008e20900030e82b0013e807000000e0001a
:1063200013003a00b6cbbf000004e00004003a00be
:10633000405f800001002000805f8800915f88003e
:10634000805f8000915f80006e014700809fbe00eb
:10635000e0122c00801f7800020078001ae8070085
:10636000e68757006e0047009cf807004900370099
:106370008e209000c0e82b00fbe707000000e00043
:1063800013003a00b6cbbf000004e00004003a005e
:10639000505f800001002000605f8800715f88000e
:1063a000605f8000715f80006e014700809fbe00cb
:1063b000f0132c00801f78000200780002e807002c
:1063c000e68757006e00470084f807003100370069
:1063d0008e20900050e92b00e3e707000000e0006a
:1063e0000c003a006e0147000000200001f8230075
:1063f000809fbe0020152c00801f780002007800ce
:10640000f1e70700e68757006e00470073f80700c2
:10641000200037008e209000e0e92b00d2e7070033
:106420000000e00002003a001c00070019003700dd
:106430008e20900070ea2b00cbe707000000e00000
:1064400014003a00b6cbbf00e14f500009003a00fb
:106450006e00470051162c001d00090031587800cd
:10646000e001b100e101b1006e0047005bf80700f8
:10647000080037006e00470031182c001d0009008d
:1064800031587800e001b100e101b1006e00470031
:1064900052f807000080fa00000006006400fa00cd
:1064a000881f7800dff80700e14f50000e003a0027
:1064b000e0f807000084fb00e1f807000080fb0023
:1064c000881f7800801f7800101a2c00801f780029
:1064d0000e007800bce70700e68757000e00780042
:1064e0003ef8070021003700d8f80700e14f5000c0
:1064f00003003200d9f80700e14f50000e003a00c7
:10650000ccf807000084fb00cdf807000080fb00fa
:10651000881f7800801f7800801e2c00801f780064
:106520000e007800a8e70700e68757000e00780005
:106530002af807000d003700bef807000084fb00b2
:10654000bff807000080fb00881f7800801f7800dc
:1065500050232c00801f78000e0078009ae7070077
:10656000e68757000e0078001cf807004f047800fb
:106570000080fa00000006000000fa0043fe070059
:10658000fccbbf00e74f500001003c00f0030700c8
:106590000080fa00000006001800fa00100f9800b2
:1065a000e800470010282c00904878001041900027
:1065b000924098006000b8006011b8005007980041
:1065c0006107980072079800030f98000040eb00e5
:1065d000404798000040eb00104798000040eb0057
:1065e000004f78001e089000e800470087e707008a
:1065f000300798003e0090000000e00003003a00e1
:1066000080002000300f9800b40137003e00900059
:10661000104078000000fb00200f9800300520009b
:10662000ae089000808f5000250132004005200008
:106630002e099000800f51000500320070042000e8
:10664000ae089000808f5000fa003200a1013700a0
:1066500004c8a90004e8a900e80047000000eb0016
:106660006ae70700300798003e0090000000e00055
:1066700003003a0072002000320f980097013700a3
:106680003e0090009040780030c5b30080cf5000ad
:1066900002003a000488a9000a0037003e0090007a
:1066a0009040780080c5b30080cf500002003a00cf
:1066b0000488a8000300370090002000300f9800e5
:1066c00086013700e80047000000eb004fe70700b5
:1066d000300798003e0090000000e00003003a0000
:1066e00071002000310f98007c0137003e009000bf
:1066f0009040780000c3b30080cf500009003a00fa
:106700003e0090000000e8009040780080c5b30093
:1067100080cf500003003a0000c1b300204798002a
:1067200002003700a0c0b300204798003e00900050
:106730006a014700ae4090006b01070030479800a7
:106740003e409000e14f500003003a00120020004c
:10675000320f9800610137005e009000ee0090005b
:106760007e0190008e099000004088001140880052
:106770005e029000ee0290007e0390008e0b90006f
:10678000f07f2000010020006011b8000020e1002f
:1067900001a8e10002b0e10003b8e1000700340005
:1067a00020408000700060000000e00003003a001c
:1067b00050002000300f9800480137005e02900022
:1067c000ee0290007e0390008e0b9000f07f200080
:1067d000010020006011b8000020e10001a8e100e4
:1067e00002b0e10003b8e10007003c002040800057
:1067f000700060000000e00003003200d1002000c3
:10680000310f980035013700e80047000000eb0029
:10681000fee60700300798003e00900090407800a8
:10682000e0c4b30080cf500008003a003e00900062
:106830000000e00003003a0072002000320f9800d0
:106840002601370004a8a9000c0037003e00900084
:106850009040780020c5b30080cf500004003a007b
:1068600010c0b3004047980004a8a80003003700f8
:10687000a0002000300f980018013700e800470002
:106880000000eb00e1e60700300798003e009000b2
:106890000000e00006003a004e4090000004e000d6
:1068a00003003a0071002000310f98000b013700ff
:1068b0006000b8006011b8005007980061079800a8
:1068c00072079800030f98003e0090006a0147008d
:1068d000a1c0b30004010700304798003e4090007b
:1068e000e14f50000c0032005e029000ee0290007a
:1068f0007e0390008e0b900080002000010020009d
:106900006011b8000020e10001a8e10002b0e10040
:1069100003b8e1000300340062002000320f980049
:10692000ee0037005e009000ee0090007e019000c7
:106930008e0990006f4060000080fb006f016000d6
:106940002140800000ff2f000080600002007000e6
:1069500020408800e80047000000eb00abe607009d
:10696000300798003e0090000000e00006003a006a
:106970004e4090000004e00003003a007000200048
:10698000300f9800d50037003e009000904078000e
:1069900000c3b30080cf500009003a003e009000d1
:1069a0000000e8009040780080c5b30080cf500020
:1069b00003003a0000c1b3002047980002003700ee
:1069c000a0c0b300204798006000b8006011b80074
:1069d000500798006107980072079800030f98000d
:1069e0003e0090006a014700ae409000be000700e4
:1069f000304798003e409000e14f500003003a00bd
:106a000021002000310f9800b40037005e00900094
:106a1000ee0090007e0190008e09900064802000be
:106a2000009abe000292be000001eb00320f9800f7
:106a3000aa00370004c8a80004e8a900e80047003d
:106a40000000eb0071e60700300798000040eb0003
:106a5000104798001e4090000081fb003e0090000f
:106a60001040780080407800e08020000000410065
:106a7000014878001e4090000040e8001047980050
:106a80003e0090000000e800300798003e009000b3
:106a9000104078000004e000eeff3a001e40900035
:106aa0008080fb00e0802000808040000040eb0000
:106ab000804878000000eb00300f98008700370016
:106ac00004c8a90004e8a800e80047000000eb00a3
:106ad0004ee60700300798000040eb00004f7800ba
:106ae0001e81fb003e00900010407800804078003e
:106af000e080200000004100014878001e4fe800bf
:106b00003e0090000000e800300798003e00900032
:106b1000104078000004e000f1ff3a009e80fb0086
:106b2000e0802000808040000040eb00804878003a
:106b3000e80047000000eb0034e60700300798004b
:106b40003e0090000000e00020003a00e1802000bc
:106b5000a0e72b0004e607000000e00003003a0075
:106b600071002000310f98005c003700e1802000a8
:106b700030e82b00fce507000000e00003003a00cd
:106b800072002000320f980054003700e18020008e
:106b9000c0e82b00f4e507000000e00003003a0025
:106ba00070002000300f98004c003700e18020007a
:106bb00070ea2b00ece507000000e00003003a005b
:106bc00071002000310f9800440037003e00900013
:106bd0009040780000c3b30080cf500009003a0015
:106be0003e0090000000e8009040780080c5b300af
:106bf00080cf500003003a0000c1b3002047980046
:106c000002003700a0c0b300204798003e0090006b
:106c10006a014700ae4090003300070030479800fb
:106c20003e409000e14f500003003a003200200047
:106c3000320f9800290037005e009000ee009000af
:106c40007e0190008e09900000408800114088006d
:106c5000e1802000a0e72b00c3e507000000e00072
:106c60000a003a00024080001340800060002000cb
:106c700001002000800f5100818f59001200360062
:106c8000b0002000300f980014003700e180200091
:106c900070ea2b00b4e507000000e0000a003a00ab
:106ca00002408000134080001000200001002000fe
:106cb000800f5100818f590003003600c100200071
:106cc000310f9800050037000001eb00320f9800eb
:106cd0000200370040002000300f98003e0890006e
:106ce0000080fa00000006001800fa00889fbe002d
:106cf0008a9fbe00000f980021579800220f98002d
:106d00006000b8006011b8001007980021079800d3
:106d100032079800430798000040eb00004f7800ce
:106d20000e089000500798000e08900090407800e0
:106d300000c3b30080cf500093003a000e089000cb
:106d40000000e8009040780080c5b30080cf50007c
:106d50008d003a0030c0b300104798000e08900034
:106d60000080e800000f98000c0037000e0890002b
:106d7000104078000080fb00c0e507000000e00044
:106d800003003a0014002000340f9800eb01370094
:106d90000e0890000000e800000f98000e08900018
:106da000104078000004e000f0ff3a00de0290009e
:106db000050f98000e0890000080e80090407800d1
:106dc0006c00470001487800ec0047000040eb00f1
:106dd000904098000e08900063004000104078003a
:106de0000004e0000c003a002e5090000081fb00ef
:106df0006c0047008000eb00aee50700100798002c
:106e0000210798004f88de00cf80de003007980011
:106e1000400798007a0137000e0890006300400098
:106e2000904078006e00470001487800ee0047006f
:106e30000040eb00904098002e5090000081fb0035
:106e40006c0047008000eb009ae507000003be00dd
:106e50002e5090000081fb00030020000234b80097
:106e600003b0b90009027800000242000790b9009f
:106e700000024200840478002e5090000081fb0044
:106e80006e0047008000eb008ae507000800400024
:106e90008980480010079800210798004f88de007d
:106ea000cf80de0030079800400798001e40900019
:106eb0000080fb00800078000e0890000100400078
:106ec000000f98002a0037000e0890000000e8002c
:106ed000904078006e00470001487800ee004700bf
:106ee0000040eb00904098002e5090000080fb0086
:106ef0000100200002002000030020001e0290007c
:106f0000ae0290003e039000ce03900022f10700f5
:106f10000205be000004be002e5090000081fb0060
:106f20006e0047008000eb0062e507000002be0033
:106f30004fabde00cfb3de000400be0006017800d8
:106f40008601780008004000898048000a01490055
:106f50008b8149001007980021079800320798009c
:106f6000430798000e0890000000e800000f98000a
:106f70000e0890000000e800104078000004e000d7
:106f8000d1ff3a001e0137000e08900090407800b3
:106f9000d0c2b30080cf500090003a0020c0b300b0
:106fa0001047980010c0b300004f78000e08900002
:106fb0000000e800000f98000d0037000e08900058
:106fc000104078008080fb0000fd2f000080400012
:106fd000e90f50000300360016002000360f98001d
:106fe000560137000e0890000000e800000f9800de
:106ff0000e089000104078000004e000efff3a0017
:10700000de039000070f98000e0890000000e800d3
:10701000904078006c00470001487800ec00470081
:107020000040eb00904098000e0890000080e800bf
:10703000104078000004e0000c003a002e50900050
:107040000081fb006c0047008000eb0019e50700a1
:1070500010079800210798004f88de00cf80de00df
:107060003007980040079800e50037000e089000b0
:107070000080e800904078006e00470001487800ea
:10708000ee0047000040eb00904098002e5090002a
:107090000081fb006c0047008000eb0005e5070065
:1070a0000003be002e5090000081fb000300200072
:1070b0000234b80003b0b9000902780000024200af
:1070c0000790b90000024200840478002e5090001e
:1070d0000081fb006e0047008000eb00f5e4070034
:1070e0000800400089804800100798002107980098
:1070f0004f88de00cf80de00300798004007980000
:107100001e4090000080fb00800078000e08900078
:1071100001004000000f98002a0037000e08900080
:107120000000e800904078006e00470001487800b9
:10713000ee0047000040eb00904098002e50900079
:107140000080fb000100200002002000030020005e
:107150001e029000ae0290003e039000ce0390000d
:107160008df007000205be000004be002e50900006
:107170000081fb006e0047008000eb00cde40700bb
:107180000002be004fabde00cfb3de000400be0045
:1071900006017800860178000800400089804800d8
:1071a0000a0149008b8149001007980021079800c7
:1071b00032079800430798000e0890000000e8008e
:1071c000000f98000e0890000000e80010407800c2
:1071d0000004e000d1ff3a008900370010c0b3007e
:1071e000104798000d0037000e08900010407800fe
:1071f0008080fb0000fd2f0000804000e90f500060
:107200000300360010002000300f9800cb0037003c
:107210000e0890000000e800000f98000e08900093
:10722000104078000004e000efff3a005e0290009a
:10723000040f98000e089000904078006c00470002
:1072400001487800ec0047000040eb0090409800b7
:107250000e0890000000e800104078000004e000f4
:107260000c003a002e5090000081fb006c0047009b
:107270008000eb008fe407001007980021079800ba
:107280004f88de00cf80de0030079800400798006e
:107290005b0037000e0890000000e8009040780086
:1072a0006e00470001487800ee0047000040eb0008
:1072b000904098002e5090000081fb006c00470029
:1072c0008000eb007be407000003be002e5090001e
:1072d0000081fb00030020000234b80003b0b900b5
:1072e00009027800000242000790b9000002420043
:1072f000840478002e5090000081fb006e0047004f
:107300008000eb006be40700080040008980480023
:1073100010079800210798004f88de00cf80de001c
:1073200030079800400798001e4090000080fb0046
:10733000800078000e08900001004000000f9800c7
:107340002a0037000e0890000000e8009040780006
:107350006e00470001487800ee0047000040eb0057
:10736000904098002e5090000080fb00010020000b
:1073700002002000030020001e029000ae029000d8
:107380003e039000ce03900003f007000205be000c
:107390000004be002e5090000081fb006e004700ec
:1073a0008000eb0043e407000002be004fabde00ac
:1073b000cfb3de000400be0006017800860178002d
:1073c00008004000898048000a0149008b8149007b
:1073d000100798002107980032079800430798008b
:1073e0000e0890000000e800000f98000e089000c2
:1073f0000000e800104078000004e000d1ff3a00ef
:107400001e029000ae0290003e039000ce0390005a
:107410006000b800020020000300280004026000a1
:107420008582600006036100878361000480ea00b2
:107430008580ea000681ea008781ea0014002000c6
:10744000050020006033b8000400e1000588e10079
:107450000690e1000798e10020003a001e0290002b
:10746000ae0290003e039000ce0390006000b80092
:1074700002002000030027000402600085826000f3
:1074800006036100878361000480ea008580ea00ca
:107490000681ea008781ea00f4ff2f00f5ff2f0044
:1074a0000403be00bcef07000203be000002be00e2
:1074b000f0ff2f00f1ff2f000001be00040040008c
:1074c000858048000601490087814900100798001f
:1074d00021079800320798004307980015c0b300b1
:1074e0009ecf12000c003a00f4ff2f00f5ff2f0092
:1074f0000403be001e009000ae0090003e0190000c
:10750000ce019000a4ef0700100798002107980013
:1075100032079800430798002e0890001e02900042
:10752000ae0290003e039000ce0390000498be008f
:107530000690be008002eb00350f98003e089000d8
:107540004f05be004f04be000080fa000000060098
:107550000200fa00889fbe00fbcbbf000080fb004a
:107560007e00b900e4004000e0812000008040007f
:10757000100078004600de00634060000080fb00e1
:10758000000f78001e007800e10f5000420032002a
:107590001e007800e20f5000470032001e00780005
:1075a0000000e0000100320051003700fbcbbf00bb
:1075b0000080fb007e00b900e6004000e081200072
:1075c000008040003002be002003be00fbcbbf00a5
:1075d0000080fb007e00b900e4004000e081200054
:1075e00000804000100078006f4060000044780088
:1075f000fbcbbf000080fb007e00b900e400400030
:10760000e081200000804000100078004500de008e
:107610006140600080447800fbcbbf000080fb002d
:107620007e00b90080007800e081200000804000ea
:107630001001be00fbcbbf000080fb007e00b90044
:10764000e4004000e081200000804000100078004d
:107650004400de0061406000849fbe00869fbe0043
:1076600008427800894078002cf70700e887570027
:1076700030282c00d9f30700f8cbbf00e14f5000b1
:107680001b003a008f60a9000040eb00f8ebb70048
:107690008f60a80016003700fbcbbf000080fb0006
:1076a0007e00b900ee004000e08120000080400034
:1076b000c6fa07000e003700fbcbbf000080fb00be
:1076c0007e00b90080007800e0812000008040004a
:1076d0001001be00fbcbbf000080fb007e00b900a4
:1076e000ee004000e08120000080400080fa0700aa
:1076f000fbcbbf000040e800fbebb700fbcbbf00bb
:10770000e84f500002003a000040eb00fbebb700ee
:107710008d20a900fccbbf000040e800fcebb700c7
:107720008d20a8004f04be000080fa000000060073
:107730000600fa00000f7800110798002207980051
:107740001e0078009e009000010878001e0078005e
:10775000ae009000110098009e0078000000eb0041
:10776000b00098009e0078000000eb00a000980098
:107770000080fa00000006000400fa0010079800dc
:107780000040eb00004f78001e00900020009000a9
:107790000000e0001e0032001e0090009000780003
:1077a0001e009000300090000080400010407800e3
:1077b000004f78001e009000300090008000e8002c
:1077c0001e009000310098001e009000b000900054
:1077d0001e00900010009000808f500007003900bc
:1077e0001e009000b00090001e009000100090005d
:1077f000808050001e009000310098001e00900014
:10780000200090008000e9001e00900021009800f8
:107810001e80fb000080fa00000006000400fa0051
:10782000000f7800110798001e007800a00090005b
:107830001e009000808f50001a0036001e00780055
:10784000b00090001e009000808040001e00780074
:10785000310098001e007800b00090001e007800f3
:1078600010009000808f5000070039001e00780043
:10787000b00090001e007800100090008080500042
:107880001e007800310098001e007800a0009000d3
:107890001e009000808050001e007800210098009b
:1078a000030037009e0078000000eb00a000980065
:1078b0000080fa00000006000400fa00000f7800c3
:1078c000110798001e007800a00090001e00900094
:1078d000808f5000070036001e007800a000900046
:1078e0001e009000808050001e007800210098004b
:1078f000030037009e0078000000eb00a000980015
:107900000080fa00000006000600fa001007980048
:10791000210798001e009000900178001e00900042
:10792000b00090002e009000808040001e0090006b
:1079300010019000110009008280d8008000fd0035
:107940000080410010407800004f78001e80fb004e
:107950000080fa00000006000600fa00000f780020
:10796000214798001e007800a00090001e007800bb
:1079700010009000808f5000170031001e0078002a
:10798000900178001e007800b00090001e00780082
:1079900020009000808040001e00780010019000c0
:1079a000110009008280d8008000fd008080410025
:1079b0002e409000804878001e0078002000900043
:1079c0008000e8001e0078002100980010002000d0
:1079d00020079800020037000000eb002007980005
:1079e0002e0090000080fa00000006000400fa005b
:1079f000100798001e009000900090001e0090005c
:107a000020009000008f50001e0078000080fa00d7
:107a1000000006000200fa00000f78009e007800c7
:107a20000000eb00a00098000080fa0000000600b3
:020000040000fa
:0200000401f009
:04000000ffff0000fe
:020000040000fa
:0200000401f009
:04000400ff7f00007a
:020000040000fa
:0200000401f009
:040008007cff000079
:020000040000fa
:0200000401f009
:04001400ffff0000ea
:020000040000fa
:100008007a4400007a4400007a4400007a440000f0
:100018007a4400007a4400007a4400007a440000e0
:100028007a4400007a4400007a4400003624000034
:100038007a4400007a4400007a4400007a440000c0
:100048007a440000f02e00007a4400007a44000050
:100058007a4400007a4400007a4400007a440000a0
:100068007a4400007a4400007a4400007a44000090
:100078007a4400007a4400007a4400007a44000080
:100088007a4400007a4400007a4400007424000096
:100098007a4400007a4400007a4400007a44000060
:1000a8007a4400007a4400007a4400007a44000050
:1000b8007a4400007a4400007a4400007a44000040
:1000c8007a4400007a4400007a4400007a44000030
:1000d8007a4400007a4400007a4400007a44000020
:1000e8007a4400007a4400007a4400007a44000010
:0800f8007a4400007a44000084
:020000040000fa
:100108007a4400007a4400007a4400007a440000ef
:100118007a4400007a4400007a4400007a440000df
:100128007a4400007a4400007a4400003624000033
:100138007a4400007a4400007a4400007a440000bf
:100148007a440000f02e00007a4400007a4400004f
:100158007a4400007a4400007a4400007a4400009f
:100168007a4400007a4400007a4400007a4400008f
:100178007a4400007a4400007a4400007a4400007f
:100188007a4400007a4400007a4400007424000095
:100198007a4400007a4400007a4400007a4400005f
:1001a8007a4400007a4400007a4400007a4400004f
:1001b8007a4400007a4400007a4400007a4400003f
:1001c8007a4400007a4400007a4400007a4400002f
:1001d8007a4400007a4400007a4400007a4400001f
:1001e8007a4400007a4400007a4400007a4400000f
:0801f8007a4400007a44000083
:020000040000fa
:107a300030780000256c000058200000256300000d
:107a40000a0d000000300000782500006c5800008e
:107a50002025000063200000257500002030000074
:107a6000782500006c6c0000580a00000d00000032
:107a70005b450000313700005d20000048610000d8
:107a8000726400007761000072650000204300000e
:107a9000414e000020720000656300006570000028
:107aa000746900006f6e00002062000075660000bf
:107ab00066650000722000006f76000065720000ad
:107ac000666c00006f7700002e2000004d650000fe
:107ad00073730000616700006520000068610000aa
:107ae0007320000062650000656e0000206c0000dd
:107af0006f730000742100000a0d0000005b00009d
:107b000045310000385d0000205300006f66000022
:107b1000747700006172000065200000434100009e
:107b20004e20000046490000464f0000206f000034
:107b300076650000726600006c6f0000772e000012
:107b4000204d000065730000736100006765000050
:107b5000206800006173000020620000656500007d
:107b60006e2000006c6f000073740000210a00009a
:107b70000d0000005b450000313900005d20000071
:107b80004d65000073730000616700006520000010
:107b90006e6f00007420000074720000616e0000bf
:107ba000736d00006974000074650000642e0000ad
:107bb000204300006f6d00006d7500006e690000cd
:107bc00063610000746900006f6e000020660000b1
:107bd000616900006c650000642e00000a0d000061
:107be0000020000020200000202000002043000092
:107bf00068650000636b0000206300006f6d00008b
:107c00006d7500006e69000063610000746900001a
:107c10006f6e00002070000061720000616d000056
:107c2000657400006572000073200000626500004a
:107c3000666f00007265000020720000657400002d
:107c400072790000696e000067200000746800000f
:107c50006520000074720000616e0000736d00000a
:107c600069730000736900006f6e00002e0a000047
:107c70000d00000020200000202000002020000037
:107c8000526500007365000074200000616c000004
:107c90006c200000434100004e200000646500009d
:107ca000766900006365000073200000746f0000b7
:107cb00020720000656300006f76000065720000ae
:107cc000206e00006f7200006d6100006c200000eb
:107cd0006f7000006572000061740000696f000041
:107ce0006e2000006d6f0000646500002e0a000029
:107cf0000d000000424100005544000052410000c8
:107d000054450000004d0000415300004b000000ae
:107d10000000000000000000464900004c54000034
:107d200045520000000000000056000045520000cf
:107d3000534900004f4e0000000000004552000073
:107d4000524f00005253000000000000004d0000a0
:107d5000455300005341000047450000000000006b
:107d60000000000001000000080000000500000005
:107d700002000000010000000500000003000000f8
:107d800005000000010000000500000003000000e5
:107d900007000000010000000800000005000000ce
:107da0001c000000010000000500000003000000ae
:107db000210000000500000008000000080000008d
:107dc0003a00000008000000080000000800000061
:107dd0000d0a00002a2a00002a2a00002a2a000090
:107de0002a2a00002a2a000042720000696400006a
:107df0006765000020430000414e0000202d000078
:107e00002052000053320000333200002f55000092
:107e100053420000206200006173000065640000ae
:107e2000206f00006e200000694300004d34000008
:107e30003031000031200000563100002e300000ab
:107e40002a2a00002a2a00002a2a00002a2a0000e2
:107e50002a2a00002a0d0000000d00000a2a000056
:107e60002a2a00002a2a00002a2a00002a2a0000c2
:107e70002a2a00002a2a00002a2a00002a2a0000b2
:107e80002a2a00002a2a00002a280000432900008c
:107e9000206900006e670000656e000069610000e7
:107ea0002d63000061740000205300002e4c000080
:107eb0002e2a00002a2a00002a2a00002a2a00006e
:107ec0002a2a00002a2a00002a2a00002a2a000062
:107ed0002a2a00002a2a00002a2a00002a2a000052
:107ee0000d0000002a2a00002a2a00002a2a000089
:107ef0002a2a00002a2a00002a2a00002a2a000032
:107f00002a2a00002a2a00002a2a00002a2a000021
:107f100077770000772e0000696e0000676500002b
:107f20006e690000612d000063610000742e000086
:107f3000636f00006d2a00002a2a00002a2a000030
:107f40002a2a00002a2a00002a2a00002a2a0000e1
:107f50002a2a00002a2a00002a2a00002a2a0000d1
:107f60002a2a00002a0d00000a0d00000a0d000058
:107f7000000000005b450000325d0000205300005f
:107f80006f660000747700006172000065200000d9
:107f900055410000525400002046000049460000b0
:107fa0004f2000006f76000065720000666c0000d4
:107fb0006f7700002e2000004d65000073730000f5
:107fc0006167000065200000686100007320000008
:107fd00062650000656e0000206c00006f73000099
:107fe000742100000a0d0000005b00004531000014
:107ff0005d200000486100007264000077610000ad
:10800000726500002055000041520000542000001d
:1080100046490000464f0000206f000076650000d2
:10802000726600006c6f0000772e0000204d00008b
:108030006573000073610000676500002068000040
:108040006173000020620000656500006e20000082
:108050006c6f000073740000210a00000d00000026
:108060000a0d00005b450000325d00002053000057
:108070006f660000747700006172000065200000e8
:1080800055410000525400002046000049460000bf
:108090004f2000006f76000065720000666c0000e3
:1080a0006f7700002e2000004d6500007373000004
:1080b0006167000065200000686100007320000017
:1080c00062650000656e0000206c00006f730000a8
:1080d000742100000a0d0000000a00000d000000dd
:1080e0000a0d0000424100005544000052410000ca
:1080f00054450000203d0000203100004d6200008a
:108100007073000020280000302900000a0d0000d4
:10811000000a00000d4200004155000044520000da
:1081200041540000452000003d2000003530000093
:10813000302000006b6200007073000020280000f7
:10814000312900000a0d0000000a00000d42000065
:1081500041550000445200004154000045200000f9
:108160003d20000032350000302000006b6200002e
:108170007073000020280000322900000a0d000062
:10818000000a00000d42000041550000445200006a
:1081900041540000452000003d2000003132000025
:1081a000352000006b620000707300002028000082
:1081b000302900000a0d0000000a00000d420000f6
:1081c0004155000044520000415400004520000089
:1081d0003d20000035300000206b00006270000080
:1081e0007320000028320000290a00000d00000062
:1081f0000a0d0000424100005544000052410000b9
:1082000054450000203d00002032000030200000d6
:108210006b6200007073000020280000332900000a
:108220000a0d0000000a00000d4200004155000048
:108230004452000041540000452000003d20000051
:1082400031300000206b00006270000073200000dd
:1082500028340000290a00000d0000000a0d00006b
:108260004d410000534b0000203d00002030000035
:10827000782500006c5800000a0d0000000a00007c
:108280000d460000494c00005445000052200000fb
:108290003d20000030780000256c0000580a0000e6
:1082a0000d0000000a0d000056450000525300006a
:1082b000494f00004e2000003d200000252e000008
:1082c000326600000a0d0000000a00000d4d00009b
:1082d0004553000053410000474500002046000080
:1082e000494c000054450000522000003d20000091
:1082f00045580000544500004e440000454400002d
:108300000a0d0000000a00000d4d0000455300005a
:10831000534100004745000020460000494c000042
:1083200054450000522000003d200000535400003e
:10833000414e000044410000524400000a0d00007c
:10834000000a00000d450000525200004f5200008c
:10835000204d00004f440000453a0000202000005e
:108360002020000020200000425500005320000083
:108370004f460000460a00000d5200005820000041
:1083800045520000524f000052200000434f0000b1
:10839000554e0000543a00002020000025750000d2
:1083a0000a0d000054580000204500005252000001
:1083b0004f520000204300004f5500004e54000073
:1083c0003a20000020250000750a00000d00000082
:1083d0000a0d000045520000524f000052200000dc
:1083e0004d4f0000444500003a20000020200000ce
:1083f0002020000020450000525200004f52000093
:108400002050000041530000534900005645000031
:108410000a0d000052580000204500005252000092
:108420004f520000204300004f5500004e54000002
:108430003a20000020250000750a00000d540000bd
:108440005820000045520000524f0000522000000a
:10845000434f0000554e0000543a00002020000019
:10846000257500000a0d0000000a00000d450000ff
:10847000525200004f520000204d00004f440000b7
:10848000453a0000202000002020000020200000ad
:1084900045520000524f00005220000041430000ae
:1084a00054490000564500000a0d000052580000d3
:1084b00020450000525200004f52000020430000af
:1084c0004f5500004e5400003a20000020250000c7
:1084d000750a00000d5400005820000045520000ad
:1084e000524f000052200000434f0000554e000044
:1084f000543a000020200000257500000a0d0000fd
:0c85000000200000000d00000a00000038
:020000040000fa
:10850c00b60b000044000000020000000100000057
:10851c000800000000000000000000000000000047
:10852c00000000000000000000000000000000003f
:10853c00000000000000000000000000000000002f
:10854c00000000000000000000000000000000001f
:10855c00000000000000000000000000000000000f
:10856c0000000000000000009e0a000086000000d1
:10857c0000000000fa0b00003200000002000000b6
:10858c0000000800000000000000000000000000d7
:10859c0000000000000000000000000000000000cf
:1085ac0000000000000000000000000000000000bf
:1085bc0000000000000000000000000000000000af
:1085cc00000000000008000016020000000000007f
:1085dc00b20c0000020000000200000000000000cd
:1085ec006a0c00000200000002000000b20c000047
:1085fc006c0c00000200000000000000160a0000d5
:10860c008800000002000000760a4e000a260a00cc
:10861c000000000000000000000000000002080044
:10862c0002024c000a4d0a004c0a4c000a4c0a008b
:10863c004c0a3c000a000000000000000000000092
:10864c00000000000000000000000000000000001e
:10865c000000020008010100740a75000a740a0087
:10866c00740a74000a740a00640a00000000000016
:10867c0000000000000000000000000000000000ee
:10868c00000000000000000001000000009c0a0037
:10869c009d0a9c000a9c0a009c0a9c000a8c0a00f9
:1086ac0000000000000000000000000000000000be
:1086bc0000000000000000000000000000000000ae
:1086cc004e0c00001200000002000000010002002d
:1086dc00000400000800100000000000202b2d00fa
:1086ec0023300000aa0c000008000000020000006b
:1086fc00686a6c00747a4c0000000000240b0000c7
:10870c004a000000020000000000210015110e00bc
:10871c000d0c0b000b0a0a000909090009090800d5
:10872c0008080800080808000707070007070700e3
:10873c000707070007070700073031003233340002
:10874c00353637003839610062636400656667004e
:10875c0068696a006b6c6d006e6f700071727300eb
:10876c0074757600777879007a000000660c00004a
:10877c0004000000020000000000000000000000e7
:10878c002c0c0000220000000200000030313200ee
:10879c003334350036373800396162006364650064
:1087ac00660030003132330034353600373839004a
:1087bc00414243004445460000000000600c0000ac
:1087cc000600000002000000000200000000000093
:1087dc006e0c000002000000000000006e0b000098
:1087ec004800000002000000000000000000000033
:1087fc002440000000000000000059004000000070
:10880c000000000088c34000000000000084d70076
:10881c009741000080e0370079c3410043176e0098
:10882c0005b5b500b8934600f5f93f00e9034f00d4
:10883c00384d32001d30f900487782005a3cbf0099
:10884c00737fdd004f157500780c000032000000be
:10885c00020000004e414e00006e61006e004900a7
:10886c004e460000696e6600003031003233340031
:10887c003536370038396100626364006566000084
:10888c00303132003334350036373800394142004c
:10889c004344450046000000700c0000020000003c
:1088ac000200000000000000b40c000002000000f8
:1088bc000200000030000000720c000002000000fa
:1088cc000200000000000000740c00000200000018
:1088dc000200000001000000760c00000200000005
:0888ec00000000000000000084
:020000040000fa
:0488f4000000fe0082
:00000001FF
